:020000040000FA
:0408000044EF08F0C9
:1008100003B213EF05F0F2B431EF05F09EB039EFFB
:1008200005F09EB241EF05F0F2A81AEF04F0F2B223
:1008300025EF04F0F2A620EF04F0F2B022EF04F06E
:10084000F3EF07F0F296F290FF00CD90F2929EA0A7
:100850002FEF04F00101533F2FEF04F0542BAEC1F2
:10086000B2F1AFC1B3F1B0C1B4F1B1C1B5F1AAC138
:10087000AEF1ABC1AFF1ACC1B0F1ADC1B1F1A6C148
:10088000AAF1A7C1ABF1A8C1ACF1A9C1ADF1A2C158
:10089000A6F1A3C1A7F1A4C1A8F1A5C1A9F19EC168
:1008A000A2F19FC1A3F1A0C1A4F1A1C1A5F19AC178
:1008B0009EF19BC19FF19CC1A0F19DC1A1F196C188
:1008C0009AF197C19BF198C19CF199C19DF1CECF4E
:1008D00096F1CFCF97F153C198F154C199F1CF6AF6
:1008E000CE6A0101536B546B9E90CD800FBC0F8E6E
:1008F0000FBA7EEF04F00F8AF3EF07F00F8C0FBEF4
:10090000BAEF04F096C19AF197C19BF198C19CF19E
:1009100099C19DF19AC19EF19BC19FF19CC1A0F12B
:100920009DC1A1F19EC1A2F19FC1A3F1A0C1A4F1FB
:10093000A1C1A5F1A2C1A6F1A3C1A7F1A4C1A8F1CB
:10094000A5C1A9F1A6C1AAF1A7C1ABF1A8C1ACF19B
:10095000A9C1ADF1AAC1AEF1ABC1AFF1ACC1B0F16B
:10096000ADC1B1F1AEC1B2F1AFC1B3F1B0C1B4F13B
:10097000B1C1B5F101015E6B5F6B606B616B96514C
:100980005E2797515F2398516023995161239A51B3
:100990005E279B515F239C5160239D5161239E5193
:1009A0005E279F515F23A0516023A1516123A25173
:1009B0005E27A3515F23A4516023A5516123A65153
:1009C0005E27A7515F23A8516023A9516123AA5133
:1009D0005E27AB515F23AC516023AD516123AE5113
:1009E0005E27AF515F23B0516023B1516123B251F3
:1009F0005E27B3515F23B4516023B5516123D89072
:100A00000101613360335F335E33D890010161339C
:100A100060335F335E33D8900101613360335F33FD
:100A20005E33F3EF07F00392ABB2AB98AB880301F0
:100A300003EE00F080517F0BE92604C0EFFF802B0E
:100A40008151805D700BD8A48B8200008051815D44
:100A5000700BD8A48B9281518019D8B40790F3EF12
:100A600007F0F2940101453FF3EF07F0462BF3EF57
:100A700007F09E900101533FF3EF07F0542BF3EF83
:100A800007F09E92040062A146EF05F007B498EFCC
:100A900005F007B098EF05F01EC620F61FC621F638
:100AA0001CC61EF61DC61FF61AC61CF61BC61DF672
:100AB00006C608F607C609F604C606F605C607F612
:100AC00002C604F603C605F626C628F627C629F68A
:100AD00024C626F625C627F622C624F623C625F602
:100AE0000EC610F60FC611F60CC60EF60DC60FF6A2
:100AF0000AC60CF60BC60DF62EC630F62FC631F61A
:100B00002CC62EF62DC62FF62AC62CF62BC62DF691
:100B100016C618F617C619F614C616F615C617F631
:100B200012C614F613C615F62CEC2CF0DAEC2BF0EA
:100B3000077C07ACB3EF05F0C274C2B4ADEF05F0AB
:100B4000C3CFB3F5C4CFB4F50501D890B433B333F4
:100B5000D890B433B333B4EF05F0C3CF55F1C4CF5D
:100B600056F1B4EF05F0C28207B421EF06F047C199
:100B70004BF148C14CF149C14DF14AC14EF15EC142
:100B800062F15FC163F160C164F161C165F196C159
:100B9000B6F197C1B7F198C1B8F199C1B9F19AC14D
:100BA000BAF19BC1BBF19CC1BCF19DC1BDF19EC11D
:100BB000BEF19FC1BFF1A0C1C0F1A1C1C1F1A2C1ED
:100BC000C2F1A3C1C3F1A4C1C4F1A5C1C5F1A6C1BD
:100BD000C6F1A7C1C7F1A8C1C8F1A9C1C9F1AAC18D
:100BE000CAF1ABC1CBF1ACC1CCF1ADC1CDF1AEC15D
:100BF000CEF1AFC1CFF1B0C1D0F1B1C1D1F1B2C12D
:100C0000D2F1B3C1D3F1B4C1D4F1B5C1D5F1B3C5FB
:100C1000B5F5B4C5B6F5B5C5B7F5B6C5B8F50101B6
:100C200055515B2756515C23E86A5D230E2E21EF58
:100C300006F05CC157F15DC158F15B6B5C6B5D6B9D
:100C4000078E0201002FF3EF07F03C0E006F00C18A
:100C50000CF101C10DF102C10EF103C10FF104C18C
:100C600010F105C111F106C112F107C113F108C15C
:100C700014F109C115F10AC116F10BC117F134C104
:100C800035F105012F51000AD8B4F2EF06F0050145
:100C90002F51010AD8B47CEF06F005012F51020A4A
:100CA000D8B4BDEF06F005012F51030AD8B4BDEF4B
:100CB00006F005012F51040AD8B4BDEF06F0050176
:100CC0002F51050AD8B4BDEF06F005012F51060AD1
:100CD000D8B4BDEF06F005012F51070AD8B4BDEF17
:100CE00006F005012F51320AD8B47AEF06F02F6BC7
:100CF000F2EF06F0F2EF06F00501536787EF06F01A
:100D0000546787EF06F0556787EF06F056678BEF5D
:100D100006F0F2EF06F057C500F158C501F159C5CC
:100D200002F15AC503F10101010E046F000E056FB7
:100D3000000E066F000E076F4BEC2AF000C157F54E
:100D400001C158F502C159F503C15AF50067B0EF6A
:100D500006F00167B0EF06F00267B0EF06F0036738
:100D6000F2EF06F053C557F554C558F555C559F57A
:100D700056C55AF50F88F2EF06F005013067C3EF4C
:100D800006F0F2EF06F00FBED8EF06F010A0DDEF90
:100D900006F001014767D4EF06F04867D4EF06F08C
:100DA0004967D4EF06F04A67D8EF06F0DDEF06F0AA
:100DB00007AEDDEF06F0EFEF06F00501312FF2EFA1
:100DC00006F03C0E316F302FF2EF06F00101000EFD
:100DD000626FE00E636FA50E646F010E656F050113
:100DE000306B0F880501626B33B7F8EF06F0628154
:100DF0000CC100F10DC101F10EC102F10FC103F1EF
:100E000010C104F111C105F112C106F113C107F1BE
:100E100014C108F115C109F116C10AF117C10BF18E
:100E200035C134F100C10CF101C10DF102C10EF167
:100E300003C10FF104C110F105C111F106C112F196
:100E400007C113F108C114F109C115F10AC116F166
:100E50000BC117F134C135F101018A6737EF07F093
:100E60008B6737EF07F08C6737EF07F08D673BEF45
:100E700007F06BEF07F08EC100F18FC101F190C157
:100E800002F191C103F10101010E046F000E056F23
:100E9000000E066F000E076F4BEC2AF000C18EF1BA
:100EA00001C18FF102C190F103C191F1006760EFC0
:100EB00007F0016760EF07F0026760EF07F0036774
:100EC0006BEF07F08AC18EF18BC18FF18CC190F16D
:100ED0008DC191F10F80D57ED5BE69D0D6CF47F1B7
:100EE000D7CF48F145C149F1E86AE8CF4AF11090FF
:100EF00047C100F148C101F149C102F14AC103F102
:100F000001010A0E046F000E056F000E066F000E41
:100F1000076F4BEC2AF003AF1080010154A79DEF3F
:100F200007F00F9A0F9C0F9E0101000E5E6F600E7E
:100F30005F6F3D0E606F080E616F010147BFADEF3F
:100F400007F04867ADEF07F04967ADEF07F04A6774
:100F5000ADEF07F0F288D2EF07F0F2985E6B5F6BAF
:100F6000606B616B966B976B986B996B9A6B9B6BD5
:100F70009C6B9D6B9E6B9F6BA06BA16BA26BA36B1D
:100F8000A46BA56BA66BA76BA86BA96BAA6BAB6BCD
:100F9000AC6BAD6BAE6BAF6BB06BB16BB26BB36B7D
:100FA000B46BB56BD76AD66A0101456B466B0CC151
:100FB00000F10DC101F10EC102F10FC103F110C129
:100FC00004F111C105F112C106F113C107F114C1F9
:100FD00008F115C109F116C10AF117C10BF135C1AC
:100FE00034F1F3EF07F002C0E0FF005001C0D8FF7A
:100FF0001000A6B2F9EF07F00CC0A9FF0BC0A8FFC4
:10100000A69EA69CA684F29E550EA76EAA0EA76E5B
:10101000A682F28EA694A6B20BEF08F00C2A12005C
:10102000A96EA69EA69CA680A8500C2A12000401B8
:101030002C0E826F53EC0BF046EC2BF00C5010ECA6
:1010400008F0E8CF00F10C5010EC08F0E8CF01F107
:1010500001AF30EF08F00101FF0E026FFF0E036FCA
:10106000E9EC2AF029673CEF08F00401200E826FBA
:1010700053EC0BF041EF08F004012D0E826F53EC9E
:101080000BF013EC29F01200076A0F6A106A0F01C7
:101090000D0EC16E860EC06E030EC26E0F01680E7D
:1010A000896E130E926E080E8A6E8A6AF30E936E24
:1010B0008B6A900E946EC80E10EC08F0E8CFE8FF33
:1010C0001098E8A0108810A805D00E0E156E8E0E90
:1010D000166E04D00F0E156E8F0E166EE4EC2CF00B
:1010E000F18EF19E0E6A01015B6B5C6B5D6B576B61
:1010F000586BF29A0101476B486B496B4A6B4B6B1B
:101100004C6B4D6B4E6B4F6B506B516B526B456B19
:10111000466BD76AD66A0F01280ED56EF28A9D906B
:10112000B00ECD6E01015E6B5F6B606B616B626BCD
:10113000636B646B656B666B676B686B696B536B3A
:10114000546BCF6ACE6A0F9A0F9C0F9E9D80760ECD
:10115000CA6E9D8202013C0E006FCC6A160E10EC26
:1011600008F0E8CF00F1170E10EC08F0E8CF01F11D
:10117000180E10EC08F0E8CF02F1190E10EC08F090
:10118000E8CF03F1010103AFE0EF08F046EC2BF0EC
:10119000160E0C6E00C10BF0F9EC07F0170E0C6E7A
:1011A00001C10BF0F9EC07F0180E0C6E02C10BF048
:1011B000F9EC07F0190E0C6E03C10BF0F9EC07F017
:1011C00000C18AF101C18BF102C18CF103C18DF123
:1011D00000C18EF101C18FF102C190F103C191F103
:1011E0001A0E10EC08F0E8CF00F11B0E10EC08F01E
:1011F000E8CF01F11C0E10EC08F0E8CF02F11D0E53
:1012000010EC08F0E8CF03F1010103AF36EF09F06D
:1012100046EC2BF01A0E0C6E00C10BF0F9EC07F047
:101220001B0E0C6E01C10BF0F9EC07F01C0E0C6EDE
:1012300002C10BF0F9EC07F01D0E0C6E03C10BF0B0
:10124000F9EC07F01A0E10EC08F0E8CF00F11B0ED5
:1012500010EC08F0E8CF01F11C0E10EC08F0E8CF1C
:1012600002F11D0E10EC08F0E8CF03F100C192F17D
:1012700001C193F102C194F103C195F1240EAC6E4A
:10128000900EAB6E240EAC6E080EB86E000EB06EF3
:101290001F0EAF6E0401806B816B0F01900EAB6E61
:1012A0000F019D8A0301806B816BC26B8B926CEC8A
:1012B00031F06CEC31F0880E10EC08F0E8CF00F162
:1012C000890E10EC08F0E8CF01F1010101AF81EFC8
:1012D00009F046EC2BF0880E0C6E00C10BF0F9EC17
:1012E00007F0890E0C6E01C10BF0F9EC07F0880EC7
:1012F00010EC08F0E8CF00F1890E10EC08F0E8CF10
:1013000001F100C140F601C141F602C142F603C13C
:1013100043F6C4EC34F04BEC2FF0200E10EC08F048
:10132000E8CF2FF505012F51FF0AD8A49FEF09F050
:101330002F6B200E0C6E2FC50BF0F9EC07F005019A
:10134000010E306F3C0E316F250E10EC08F0E8CF27
:1013500000F1260E10EC08F0E8CF01F1270E10EC9A
:1013600008F0E8CF02F1280E10EC08F0E8CF03F106
:10137000010103AFD6EF09F046EC2BF0250E0C6E01
:1013800000C10BF0F9EC07F0260E0C6E01C10BF05A
:10139000F9EC07F0270E0C6E02C10BF0F9EC07F028
:1013A000280E0C6E03C10BF0F9EC07F000C153F5E9
:1013B00001C154F502C155F503C156F500C157F5F9
:1013C00001C158F502C159F503C15AF5290E10ECB7
:1013D00008F0E8CF5BF505015C515B5DD8A05BC50B
:1013E0005CF505012F51020A0EE181B803EF0AF006
:1013F00005015C2F00EF0AF05BC55CF503EF0AF016
:1014000081BA03EF35F0210E10EC08F0E8CF00F1BF
:10141000220E10EC08F0E8CF01F1230E10EC08F0DA
:10142000E8CF02F1240E10EC08F0E8CF03F101013F
:1014300003AF49EF0AF046EC2BF0210E0C6E00C111
:101440000BF0F9EC07F0220E0C6E01C10BF0F9EC79
:1014500007F0230E0C6E02C10BF0F9EC07F0240E1E
:101460000C6E03C10BF0F9EC07F0210E10EC08F044
:10147000E8CF00F1220E10EC08F0E8CF01F1230EC6
:1014800010EC08F0E8CF02F1240E10EC08F0E8CFE1
:1014900003F100C15DF501C15EF502C15FF503C155
:1014A00060F593EC2EF095EC2DF0EDEC2CF00501B1
:1014B0002F51030A12E005012F51040A1DE0050116
:1014C0002F51050A24E005012F51060A32E00501DB
:1014D0002F51070A38E0ACEF0AF0ACC500F101016A
:1014E0000F0E001701010051000A36E00101005102
:1014F000050A32E0A9EF0AF0ACC500F101010F0EB8
:10150000001701010051000A27E0A9EF0AF00501C8
:10151000AC51000A21E00501AC51150A1DE005019E
:10152000AC51300A19E00501AC51450A15E0A9EFAC
:101530000AF00501AC51000A0FE00501AC51300A78
:101540000BE0A9EF0AF00501AC51000A05E0A9EF94
:101550000AF081BA03EF35F07EEC2CF00790000121
:10156000F28EF28C07B0A7EF26F00FB086EF21F0D5
:101570000FB84AEF1BF00301805181197F0BD8B4DB
:10158000A7EF26F013EE00F081517F0BE126812BAF
:10159000E7CFE8FFE00BD8B4A7EF26F023EE82F008
:1015A000C2513F0BD926E7CFDFFFC22BDF50780AAD
:1015B000D8A4A7EF26F007808EC100F18FC101F1FA
:1015C00090C102F191C103F10101040E046F000EFC
:1015D000056F000E066F000E076F4BEC2AF000AF90
:1015E000FBEF0AF00101030E8E6F000E8F6F000EED
:1015F000906F000E916F03018251720AD8B486EF8A
:1016000021F08251520AD8B486EF21F08251750A36
:10161000D8B486EF21F08251630AD8B461EF23F089
:101620008251690AD8B441EF1EF082517A0AD8B4C7
:1016300054EF1FF08251490AD8B4E0EF1DF08251F7
:10164000500AD8B4FEEF1CF08251700AD8B441EFB2
:101650001DF08251540AD8B46CEF1DF08251740A07
:10166000D8B4B2EF1DF082516D0AD8B467EF0BF019
:1016700082514D0AD8B480EF0BF08251730AD8B46E
:10168000B6EF20F08251530AD8B41BEF21F08251FB
:101690004C0AD8B4E3EF12F08251760AD8B40FEFB7
:1016A0000CF098EF23F0040114EE00F080517F0B52
:1016B000E12682C4E7FF802B120004010D0E826F29
:1016C00053EC0BF00A0E826F53EC0BF01200040186
:1016D0006D0E826F53EC0BF003018351300AD8B4C6
:1016E000BFEF0BF003018351310AD8B4D2EF0BF0F6
:1016F00003018351320AD8B4E5EF0BF098EF23F0E1
:1017000004014D0E826F53EC0BF087EC2BF084C379
:1017100031F185C332F186C333F10101296B94ECB9
:101720002BF00BEC2BF003018351300AD8B4A7EF58
:101730000BF003018351310AD8B4AFEF0BF0030172
:101740008351320AD8B4B7EF0BF098EF23F0FD0EB7
:101750000C6E00C10BF0F9EC07F0BFEF0BF0FE0EC2
:101760000C6E00C10BF0F9EC07F0D2EF0BF0FF0E9E
:101770000C6E00C10BF0F9EC07F0E5EF0BF0040183
:10178000300E826F53EC0BF004012C0E826F53EC81
:101790000BF046EC2BF0FD0E10EC08F0E8CF00F15A
:1017A000F6EF0BF00401310E826F53EC0BF00401E5
:1017B0002C0E826F53EC0BF046EC2BF0FE0E10EC6F
:1017C00008F0E8CF00F1F6EF0BF00401320E826F63
:1017D00053EC0BF046EC2BF004012C0E826F53EC13
:1017E0000BF0FF0E10EC08F0E8CF00F1E9EC2AF066
:1017F00031C182F40401300E822753EC0BF032C168
:1018000082F40401300E822753EC0BF033C182F4D2
:101810000401300E822753EC0BF096EF23F0030106
:101820008351300AD8B4B4EF0DF003018351310A6B
:10183000D8B4EBEF0DF003018351320AD8B4A0EF16
:101840000FF003018351330AD8B455EF11F00301AF
:101850008351340AD8B4FBEF11F003018351730AAA
:10186000D8B496EF0CF003018351760AD8B498EF00
:101870000CF003018351740AD8B483EF0CF0030118
:101880008351540AD8B448EF0CF0D8A498EF23F051
:101890000401760E826F53EC0BF00401540E826F3C
:1018A00053EC0BF007840001880E0C6E87EC2BF0D4
:1018B0002981030184512D0AD8B461EF0CF0010194
:1018C000299185C32FF186C330F187C331F188C3D5
:1018D00032F189C333F194EC2BF00BEC2BF000C107
:1018E0000BF0F9EC07F001C10BF0F9EC07F0880EF2
:1018F00010EC08F0E8CF40F6890E10EC08F0E8CFC5
:1019000041F68EEF0CF00401760E826F53EC0BF073
:101910000401740E826F53EC0BF007840001880EF3
:101920000C6E17EC08F00794ABEF1BF096EC0CF084
:101930000401760E826F53EC0BF00401760E826F79
:1019400053EC0BF00784C3EC27F004012C0E826FDC
:1019500053EC0BF00101036B026B3BC601F13AC67D
:1019600000F101AFB9EF0CF00101FF0E026FFF0EA5
:10197000036FE9EC2AF02967C0EF0CF0C5EF0CF01B
:1019800004012D0E826F53EC0BF02FC182F4040181
:10199000300E822753EC0BF030C182F40401300E7C
:1019A000822753EC0BF031C182F40401300E822700
:1019B00053EC0BF032C182F40401300E822753EC59
:1019C0000BF033C182F40401300E822753EC0BF08C
:1019D00004012C0E826F53EC0BF00101036B026BC0
:1019E0003DC601F13CC600F101AFFCEF0CF0010176
:1019F000FF0E026FFF0E036FE9EC2AF0296703EF79
:101A00000DF008EF0DF004012D0E826F53EC0BF07A
:101A10002FC182F40401300E822753EC0BF030C149
:101A200082F40401300E822753EC0BF031C182F4B2
:101A30000401300E822753EC0BF032C182F4040112
:101A4000300E822753EC0BF033C182F40401300EC8
:101A5000822753EC0BF004012C0E826F53EC0BF039
:101A60000101036B026B3FC601F13EC600F101AFFD
:101A70003FEF0DF00101FF0E026FFF0E036FE9EC67
:101A80002AF0296746EF0DF04BEF0DF004012D0E03
:101A9000826F53EC0BF02FC182F40401300E8227C9
:101AA00053EC0BF030C182F40401300E822753EC6A
:101AB0000BF031C182F40401300E822753EC0BF09D
:101AC00032C182F40401300E822753EC0BF033C193
:101AD00082F40401300E822753EC0BF004012C0E2B
:101AE000826F53EC0BF00101036B026B37C601F1FF
:101AF00036C600F101AF82EF0DF00101FF0E026F5B
:101B0000FF0E036FE9EC2AF0296789EF0DF08EEFE5
:101B10000DF004012D0E826F53EC0BF02FC182F4F7
:101B20000401300E822753EC0BF030C182F4040123
:101B3000300E822753EC0BF031C182F40401300ED9
:101B4000822753EC0BF032C182F40401300E82275D
:101B500053EC0BF033C182F40401300E822753ECB6
:101B60000BF00794ABEF1BF00401760E826F53EC81
:101B70000BF00401300E826F53EC0BF004012C0EBD
:101B8000826F53EC0BF0B4EC2BF046EC2BF000C65C
:101B900000F101C601F1E9EC2AF030C182F4040140
:101BA000300E822753EC0BF031C182F40401300E69
:101BB000822753EC0BF032C182F40401300E8227ED
:101BC00053EC0BF033C182F40401300E822753EC46
:101BD0000BF0ABEF1BF00401760E826F53EC0BF0B1
:101BE0000401310E826F53EC0BF007840101036B8B
:101BF000026B02C600F103C601F101AF04EF0EF063
:101C0000FF0E026FFF0E036F0101076B066B04C628
:101C100004F105C605F105AF12EF0EF0FF0E066FD9
:101C2000FF0E076F50EC2AF00101076B066B06C62A
:101C300004F107C605F105AF22EF0EF0FF0E066FA7
:101C4000FF0E076F50EC2AF00101076B066B08C608
:101C500004F109C605F105AF32EF0EF0FF0E066F75
:101C6000FF0E076F50EC2AF0D890010103330233C6
:101C700001330033D89001010333023301330033C1
:101C800004012C0E826F53EC0BF00101036B026B0D
:101C900001C101F100C100F101AF54EF0EF00101EB
:101CA000FF0E026FFF0E036FE9EC2AF029675BEF6E
:101CB0000EF060EF0EF004012D0E826F53EC0BF06E
:101CC0002FC182F40401300E822753EC0BF030C197
:101CD00082F40401300E822753EC0BF031C182F400
:101CE0000401300E822753EC0BF032C182F4040160
:101CF000300E822753EC0BF033C182F40401300E16
:101D0000822753EC0BF00101036B026B0AC600F152
:101D10000BC601F101AF91EF0EF0FF0E026FFF0E47
:101D2000036F0101076B066B0CC604F10DC605F1CC
:101D300005AF9FEF0EF0FF0E066FFF0E076F50EC22
:101D40002AF00101076B066B0EC604F10FC605F100
:101D500005AFAFEF0EF0FF0E066FFF0E076F50ECF2
:101D60002AF00101076B066B10C604F111C605F1DC
:101D700005AFBFEF0EF0FF0E066FFF0E076F50ECC2
:101D80002AF0D89001010333023301330033D89095
:101D90000101033302330133003304012C0E826F3F
:101DA00053EC0BF00101036B026B01C101F100C1A7
:101DB00000F101AFE1EF0EF00101FF0E026FFF0E27
:101DC000036FE9EC2AF02967E8EF0EF0EDEF0EF073
:101DD00004012D0E826F53EC0BF02FC182F404012D
:101DE000300E822753EC0BF030C182F40401300E28
:101DF000822753EC0BF031C182F40401300E8227AC
:101E000053EC0BF032C182F40401300E822753EC04
:101E10000BF033C182F40401300E822753EC0BF037
:101E20000101036B026B12C600F113C601F101AF91
:101E30001EEF0FF0FF0E026FFF0E036F0101076B25
:101E4000066B14C604F115C605F105AF2CEF0FF0B3
:101E5000FF0E066FFF0E076F50EC2AF00101076BB3
:101E6000066B16C604F117C605F105AF3CEF0FF07F
:101E7000FF0E066FFF0E076F50EC2AF00101076B93
:101E8000066B18C604F119C605F105AF4CEF0FF04B
:101E9000FF0E066FFF0E076F50EC2AF0D89001017D
:101EA0000333023301330033D8900101033302338B
:101EB0000133003304012C0E826F53EC0BF001014F
:101EC000036B026B01C101F100C100F101AF6EEFC4
:101ED0000FF00101FF0E026FFF0E036FE9EC2AF015
:101EE000296775EF0FF07AEF0FF004012D0E826F66
:101EF00053EC0BF02FC182F40401300E822753EC17
:101F00000BF030C182F40401300E822753EC0BF049
:101F100031C182F40401300E822753EC0BF032C140
:101F200082F40401300E822753EC0BF033C182F4AB
:101F30000401300E822753EC0BF00794ABEF1BF03B
:101F40000401760E826F53EC0BF00401320E826FA7
:101F500053EC0BF007840101036B026B1AC600F10E
:101F60001BC601F101AFB9EF0FF0FF0E026FFF0EBC
:101F7000036F0101076B066B1CC604F11DC605F15A
:101F800005AFC7EF0FF0FF0E066FFF0E076F50ECA7
:101F90002AF00101076B066B1EC604F11FC605F18E
:101FA00005AFD7EF0FF0FF0E066FFF0E076F50EC77
:101FB0002AF00101076B066B20C604F121C605F16A
:101FC00005AFE7EF0FF0FF0E066FFF0E076F50EC47
:101FD0002AF0D89001010333023301330033D89043
:101FE0000101033302330133003304012C0E826FED
:101FF00053EC0BF00101036B026B01C101F100C155
:1020000000F101AF09EF10F00101FF0E026FFF0EAA
:10201000036FE9EC2AF0296710EF10F015EF10F0CC
:1020200004012D0E826F53EC0BF02FC182F40401DA
:10203000300E822753EC0BF030C182F40401300ED5
:10204000822753EC0BF031C182F40401300E822759
:1020500053EC0BF032C182F40401300E822753ECB2
:102060000BF033C182F40401300E822753EC0BF0E5
:102070000101036B026B22C600F123C601F101AF1F
:1020800046EF10F0FF0E026FFF0E036F0101076BAA
:10209000066B24C604F125C605F105AF54EF10F018
:1020A000FF0E066FFF0E076F50EC2AF00101076B61
:1020B000066B26C604F127C605F105AF64EF10F0E4
:1020C000FF0E066FFF0E076F50EC2AF00101076B41
:1020D000066B28C604F129C605F105AF74EF10F0B0
:1020E000FF0E066FFF0E076F50EC2AF0D89001012B
:1020F0000333023301330033D89001010333023339
:102100000133003304012C0E826F53EC0BF00101FC
:10211000036B026B01C101F100C100F101AF96EF49
:1021200010F00101FF0E026FFF0E036FE9EC2AF0C1
:1021300029679DEF10F0A2EF10F004012D0E826FC1
:1021400053EC0BF02FC182F40401300E822753ECC4
:102150000BF030C182F40401300E822753EC0BF0F7
:1021600031C182F40401300E822753EC0BF032C1EE
:1021700082F40401300E822753EC0BF033C182F459
:102180000401300E822753EC0BF00101036B026B4C
:102190002AC600F12BC601F101AFD3EF10F0FF0EFC
:1021A000026FFF0E036F0101076B066B2CC604F173
:1021B0002DC605F105AFE1EF10F0FF0E066FFF0E23
:1021C000076F50EC2AF00101076B066B2EC604F175
:1021D0002FC605F105AFF1EF10F0FF0E066FFF0EF1
:1021E000076F50EC2AF00101076B066B30C604F153
:1021F00031C605F105AF01EF11F0FF0E066FFF0EBE
:10220000076F50EC2AF0D8900101033302330133F9
:102210000033D8900101033302330133003304014A
:102220002C0E826F53EC0BF00101036B026B01C1AA
:1022300001F100C100F101AF23EF11F00101FF0E28
:10224000026FFF0E036FE9EC2AF029672AEF11F005
:102250002FEF11F004012D0E826F53EC0BF02FC104
:1022600082F40401300E822753EC0BF030C182F46B
:102270000401300E822753EC0BF031C182F40401CB
:10228000300E822753EC0BF032C182F40401300E81
:10229000822753EC0BF033C182F40401300E822705
:1022A00053EC0BF00794ABEF1BF00401760E826F3A
:1022B00053EC0BF00401330E826F53EC0BF004016E
:1022C0002C0E826F53EC0BF085C382F453EC0BF0B1
:1022D000640E0D6E03018551320A02E16A0E0D6E25
:1022E00003018551330A02E1700E0D6E0301855121
:1022F000340A02E1760E0D6E03018551350A02E1C2
:102300007C0E0D6E03018551360A02E1820E0D6EC0
:1023100003018651780A65E00DC00CF087EC2BF0C4
:102320002981030187512D0AD8B499EF11F00101D9
:10233000299188C32FF189C330F18AC331F18BC34E
:1023400032F18CC333F194EC2BF00BEC2BF000C189
:102350000BF0F9EC07F001C10BF0F9EC07F087EC9A
:102360002BF0298103018E512D0AD8B4BAEF11F058
:10237000010129918FC32FF190C330F191C331F145
:1023800092C332F193C333F194EC2BF00BEC2BF0AE
:1023900000C10BF0F9EC07F001C10BF0F9EC07F00C
:1023A00087EC2BF02981030195512D0AD8B4DBEF7E
:1023B00011F00101299196C32FF197C330F198C311
:1023C00031F199C332F19AC333F194EC2BF00BEC59
:1023D0002BF000C10BF0F9EC07F001C10BF0F9ECA8
:1023E00007F00DC00CF017EC08F017EC08F017EC34
:1023F00008F0ABEF1BF00401760E826F53EC0BF08C
:102400000401340E826F53EC0BF003018451780AFF
:10241000D8B4D3EF12F03E0E0C6E87EC2BF029816E
:10242000030185512D0AD8B418EF12F0010129914A
:1024300086C32FF187C330F188C331F189C332F1EC
:102440008AC333F194EC2BF00BEC2BF000C10BF0B2
:10245000F9EC07F001C10BF0F9EC07F087EC2BF079
:10246000298103018C512D0AD8B439EF12F00101F2
:1024700029918DC32FF18EC330F18FC331F190C3F9
:1024800032F191C333F194EC2BF00BEC2BF000C143
:102490000BF0F9EC07F001C10BF0F9EC07F087EC59
:1024A0002BF02981030193512D0AD8B45AEF12F071
:1024B0000101299194C32FF195C330F196C331F1F5
:1024C00097C332F198C333F194EC2BF00BEC2BF063
:1024D00000C10BF0F9EC07F001C10BF0F9EC07F0CB
:1024E00087EC2BF0298103019A512D0AD8B47BEF98
:1024F00012F0010129919BC32FF19CC330F19DC3C0
:1025000031F19EC332F19FC333F194EC2BF00BEC0D
:102510002BF000C10BF0F9EC07F001C10BF0F9EC66
:1025200007F087EC2BF029810301A1512D0AD8B4C3
:102530009CEF12F001012991A2C32FF1A3C330F146
:10254000A4C331F1A5C332F1A6C333F194EC2BF04F
:102550000BEC2BF000C10BF0F9EC07F001C10BF014
:10256000F9EC07F087EC2BF029810301A8512D0A23
:10257000D8B4BDEF12F001012991A9C32FF1AAC36C
:1025800030F1ABC331F1ACC332F1ADC333F194ECF4
:102590002BF00BEC2BF000C10BF0F9EC07F001C1B4
:1025A0000BF0F9EC07F03E0E0C6E17EC08F017EC90
:1025B00008F017EC08F017EC08F017EC08F017EC2F
:1025C00008F0ABEF1BF003018351300AD8B44EEF93
:1025D00016F003018351310AD8B47BEF17F00301E1
:1025E0008351320AD8B4E9EF17F003018351330A5B
:1025F000D8B4F9EF17F003018351340AD8B409EFC6
:1026000018F003018351350AD8B44FEF1BF00301D2
:102610008351360AD8B47DEF1BF003018351370A8A
:10262000D8B4B0EF15F003018351460AD8B4A3EF34
:102630001AF0030183514D0AD8B429EF14F00301B5
:1026400083516D0AD8B443EF14F0030183515A0A41
:10265000D8B4F5EF16F003018351490AD8B47DEFE1
:102660001CF003018351500AD8B4AFEF1BF00301F3
:102670008351540AD8B428EF1CF003018351630A34
:10268000D8B463EF14F003018351430AD8B45BEF6D
:1026900015F003018351730AD8B461EF14F00301FC
:1026A0008351610AD8B476EF13F003018351650AB0
:1026B000D8B49EEF16F003018351450AD8B4ACEFAD
:1026C00016F003018351620AD8B4BAEF16F0030181
:1026D0008351420AD8B4C8EF16F003018351760A39
:1026E000D8B4D6EF16F0D8A498EF23F004014C0E1E
:1026F000826F53EC0BF00401610E826F53EC0BF010
:1027000095EC2DF004012C0E826F53EC0BF046EC8F
:102710002BF0ABC500F10101E9EC2AF031C182F4E4
:102720000401300E822753EC0BF032C182F4040115
:10273000300E822753EC0BF033C182F40401300ECB
:10274000822753EC0BF004012C0E826F53EC0BF03C
:1027500046EC2BF0ACC500F10101E9EC2AF031C1E7
:1027600082F40401300E822753EC0BF032C182F464
:102770000401300E822753EC0BF033C182F40401C4
:10278000300E822753EC0BF004012C0E826F53ECB9
:102790000BF046EC2BF0ADC500F10101E9EC2AF09D
:1027A00031C182F40401300E822753EC0BF032C1A8
:1027B00082F40401300E822753EC0BF033C182F413
:1027C0000401300E822753EC0BF004012C0E826FB3
:1027D00053EC0BF046EC2BF0AEC500F10101E9EC37
:1027E0002AF031C182F40401300E822753EC0BF041
:1027F00032C182F40401300E822753EC0BF033C156
:1028000082F40401300E822753EC0BF004012C0EED
:10281000826F53EC0BF046EC2BF0B2C500F10101D6
:10282000E9EC2AF031C182F40401300E822753EC26
:102830000BF032C182F40401300E822753EC0BF00E
:1028400033C182F40401300E822753EC0BF0ABEF5E
:102850001BF087EC2BF084C333F194EC2BF00BECE2
:102860002BF0200E0C6E00C10BF0F9EC07F000C14C
:102870002FF505012F51000A06E005012F51010A2D
:1028800002E02FEC2EF004014C0E826F53EC0BF0A3
:1028900004014D0E826F53EC0BF004012C0E826F7D
:1028A00053EC0BF046EC2BF02FC500F1E9EC2AF0CD
:1028B00033C182F40401300E822753EC0BF0ABEFEE
:1028C0001BF003EF35F004014C0E826F53EC0BF05C
:1028D0000401630E826F53EC0BF0EDEC2CF004015D
:1028E0002C0E826F53EC0BF078EC14F0ABEF1BF076
:1028F00046EC2BF0B1C500F10101003B0F0E0017B3
:10290000E9EC2AF033C182F40401300E822753EC43
:102910000BF0B1C500F101010F0E01010017E9EC48
:102920002AF033C182F40401300E822753EC0BF0FD
:1029300004012D0E826F53EC0BF0B0C500F10101C4
:10294000003B0F0E0017E9EC2AF033C182F40401BA
:10295000300E822753EC0BF0B0C500F101010F0ED1
:1029600001010017E9EC2AF033C182F40401300EB2
:10297000822753EC0BF004012D0E826F53EC0BF009
:10298000AFC500F10101003B0F0E0017E9EC2AF082
:1029900033C182F40401300E822753EC0BF0AFC533
:1029A00000F101010F0E01010017E9EC2AF033C11B
:1029B00082F40401300E822753EC0BF00401200E48
:1029C000826F53EC0BF0AEC500F10F0E0101001742
:1029D000E9EC2AF033C182F40401300E822753EC73
:1029E0000BF00401200E826F53EC0BF0ADC500F12B
:1029F00001010101003B0F0E0017E9EC2AF033C181
:102A000082F40401300E822753EC0BF0ADC500F1C7
:102A100001010F0E01010017E9EC2AF033C182F425
:102A20000401300E822753EC0BF004013A0E826F42
:102A300053EC0BF0ACC500F10101003B0F0E001789
:102A4000E9EC2AF033C182F40401300E822753EC02
:102A50000BF0ACC500F101010F0E01010017E9EC0C
:102A60002AF033C182F40401300E822753EC0BF0BC
:102A700004013A0E826F53EC0BF0ABC500F101017B
:102A8000003B0F0E0017E9EC2AF033C182F4040179
:102A9000300E822753EC0BF0ABC500F101010F0E95
:102AA0000017E9EC2AF033C182F40401300E8227CA
:102AB00053EC0BF0120084C3E8FF0F0BE83AE8CFA9
:102AC000B1F585C3E8FF0F0B0501B11387C3E8FF1C
:102AD0000F0BE83AE8CFB0F588C3E8FF0F0B05010C
:102AE000B0138AC3E8FF0F0BE83AE8CFAFF58BC30A
:102AF000E8FF0F0B0501AF138DC3E8FF0F0BE8CF05
:102B0000AEF58FC3E8FF0F0BE83AE8CFADF590C301
:102B1000E8FF0F0B0501AD1392C3E8FF0F0BE83A76
:102B2000E8CFACF593C3E8FF0F0B0501AC1395C3D9
:102B3000E8FF0F0BE83AE8CFABF596C3E8FF0F0BC1
:102B40000501AB1348EC2DF004014C0E826F53ECE1
:102B50000BF00401430E826F53EC0BF06DEF14F099
:102B6000078404014C0E826F53EC0BF00401370E06
:102B7000826F53EC0BF004012C0E826F53EC0BF0C0
:102B800005012E51130A06E005012E51170A0DE02A
:102B90004BEF16F00101000E006F000E016F100EDA
:102BA000026F000E036FDEEF15F00101000E006FE3
:102BB000000E016F000E026F010E036FE9EC2AF0A8
:102BC0002AC182F40401300E822753EC0BF02BC192
:102BD00082F40401300E822753EC0BF02CC182F4F6
:102BE0000401300E822753EC0BF02DC182F4040156
:102BF000300E822753EC0BF02EC182F40401300E0C
:102C0000822753EC0BF02FC182F40401300E82278F
:102C100053EC0BF030C182F40401300E822753ECE8
:102C20000BF031C182F40401300E822753EC0BF01B
:102C300032C182F40401300E822753EC0BF033C111
:102C400082F40401300E822753EC0BF004012C0EA9
:102C5000826F53EC0BF00101200E006F000E016F2C
:102C6000000E026F000E036FE9EC2AF031C182F40E
:102C70000401300E822753EC0BF032C182F40401C0
:102C8000300E822753EC0BF033C182F40401300E76
:102C9000822753EC0BF00794ABEF1BF00784C4ECD6
:102CA00034F046EC2BF02DC500F1E9EC2AF00401DC
:102CB0004C0E826F53EC0BF00401300E826F53EC1C
:102CC0000BF004012C0E826F53EC0BF031C182F437
:102CD0000401300E822753EC0BF032C182F4040160
:102CE000300E822753EC0BF033C182F40401300E16
:102CF000822753EC0BF004012C0E826F53EC0BF087
:102D000046EC2BF02EC500F1E9EC2AF031C182F43B
:102D10000401300E822753EC0BF032C182F404011F
:102D2000300E822753EC0BF033C182F40401300ED5
:102D3000822753EC0BF00794ABEF1BF004014C0E11
:102D4000826F53EC0BF00401650E826F53EC0BF0B5
:102D5000EFEC2EF0ABEF1BF004014C0E826F53EC46
:102D60000BF00401450E826F53EC0BF006EC2FF0D4
:102D7000ABEF1BF004014C0E826F53EC0BF004011F
:102D8000620E826F53EC0BF034EC2FF0ABEF1BF0C4
:102D900004014C0E826F53EC0BF00401420E826F63
:102DA00053EC0BF01DEC2FF0ABEF1BF004014C0EBD
:102DB000826F53EC0BF00401760E826F53EC0BF034
:102DC00004012C0E826F53EC0BF010A807D0040105
:102DD000310E826F53EC0BF0ABEF1BF00401300EA1
:102DE000826F53EC0BF0ABEF1BF004014C0E826FC3
:102DF00053EC0BF004015A0E826F53EC0BF00401FC
:102E00002C0E826F53EC0BF0C4EC34F046EC2BF03C
:102E100005012E51130A06E005012E51170A0DE097
:102E200026EF17F00101000E006F000E016F100E6B
:102E3000026F000E036F26EF17F00101000E006F06
:102E4000000E016F000E026F010E036F0101200ED4
:102E5000046F000E056F000E066F000E076F7CEC0E
:102E60002AF0E9EC2AF02AC182F40401300E82270C
:102E700053EC0BF02BC182F40401300E822753EC8B
:102E80000BF02CC182F40401300E822753EC0BF0BE
:102E90002DC182F40401300E822753EC0BF02EC1B9
:102EA00082F40401300E822753EC0BF02FC182F420
:102EB0000401300E822753EC0BF030C182F4040180
:102EC000300E822753EC0BF031C182F40401300E36
:102ED000822753EC0BF032C182F40401300E8227BA
:102EE00053EC0BF033C182F40401300E822753EC13
:102EF0000BF0ABEF1BF0078404014C0E826F53EC18
:102F00000BF00401310E826F53EC0BF004012C0E18
:102F1000826F53EC0BF025C500F126C501F127C5E2
:102F200002F128C503F10101200E046F000E056FA8
:102F3000000E066F000E076F7CEC2AF0E9EC2AF019
:102F40002AC182F40401300E822753EC0BF02BC10E
:102F500082F40401300E822753EC0BF02CC182F472
:102F60000401300E822753EC0BF02DC182F40401D2
:102F7000300E822753EC0BF02EC182F40401300E88
:102F8000822753EC0BF02FC182F40401300E82270C
:102F900053EC0BF030C182F40401300E822753EC65
:102FA0000BF031C182F40401300E822753EC0BF098
:102FB00032C182F40401300E822753EC0BF033C18E
:102FC00082F40401300E822753EC0BF00794ABEF30
:102FD0001BF0078404014C0E826F53EC0BF00401CC
:102FE000320E826F53EC0BF022EC31F00794ABEF12
:102FF0001BF0078404014C0E826F53EC0BF00401AC
:10300000330E826F53EC0BF07FEC31F0079486EFB8
:1030100017F0078404014C0E826F53EC0BF004018F
:10302000340E826F53EC0BF004012C0E826F53ECC4
:103030000BF087EC2BF084C32AF185C32BF186C3F8
:103040002CF187C32DF188C32EF189C32FF18AC3D8
:1030500030F18BC331F18CC332F18DC333F10101F7
:10306000296B94EC2BF00BEC2BF0200E046F000E70
:10307000056F000E066F000E076F5CEC2AF000C1B2
:1030800021F501C122F502C123F503C124F577EC36
:1030900034F034C5ABF535C5ACF536C5ADF537C53F
:1030A000AEF538C5AFF539C5B0F53AC5B1F578EC30
:1030B00014F004012C0E826F53EC0BF03BC500F1B1
:1030C0003CC501F13DC502F13EC503F10101000E11
:1030D000046F000E056F010E066F000E076F7CEC8B
:1030E0002AF0E9EC2AF0296778EF18F07DEF18F064
:1030F00004012D0E826F53EC0BF030C182F40401F9
:10310000300E822753EC0BF031C182F40401300EF3
:10311000822753EC0BF004012E0E826F53EC0BF060
:1031200032C182F40401300E822753EC0BF033C11C
:1031300082F40401300E822753EC0BF004012C0EB4
:10314000826F53EC0BF046EC2BF03FC500F140C50D
:1031500001F1C2EC24F004012C0E826F53EC0BF051
:1031600046EC2BF041C500F1E9EC2AF031C182F4C4
:103170000401300E822753EC0BF032C182F40401BB
:10318000300E822753EC0BF033C182F40401300E71
:10319000822753EC0BF004012C0E826F53EC0BF0E2
:1031A0000101036B026B48C501F147C500F101AF96
:1031B000DFEF18F00101FF0E026FFF0E036FE9EC65
:1031C0002AF02967E6EF18F0EBEF18F004012D0E56
:1031D000826F53EC0BF02FC182F40401300E822772
:1031E00053EC0BF030C182F40401300E822753EC13
:1031F0000BF031C182F40401300E822753EC0BF046
:1032000032C182F40401300E822753EC0BF033C13B
:1032100082F40401300E822753EC0BF004012C0ED3
:10322000826F53EC0BF00101036B026B4AC501F195
:1032300049C500F101AF22EF19F00101FF0E026F45
:10324000FF0E036FE9EC2AF0296729EF19F02EEF42
:1032500019F004012D0E826F53EC0BF02FC182F494
:103260000401300E822753EC0BF030C182F40401CC
:10327000300E822753EC0BF031C182F40401300E82
:10328000822753EC0BF032C182F40401300E822706
:1032900053EC0BF033C182F40401300E822753EC5F
:1032A0000BF004012C0E826F53EC0BF00101036B49
:1032B000026B4CC501F14BC500F101AF65EF19F090
:1032C0000101FF0E026FFF0E036FE9EC2AF0296780
:1032D0006CEF19F071EF19F004012D0E826F53ECB1
:1032E0000BF02FC182F40401300E822753EC0BF057
:1032F00030C182F40401300E822753EC0BF031C14F
:1033000082F40401300E822753EC0BF032C182F4B8
:103310000401300E822753EC0BF033C182F4040118
:10332000300E822753EC0BF004012C0E826F53EC0D
:103330000BF00101036B026B4EC501F14DC500F1AD
:1033400001AFA8EF19F00101FF0E026FFF0E036F2E
:10335000E9EC2AF02967AFEF19F0B4EF19F0040196
:103360002D0E826F53EC0BF02FC182F40401300E4E
:10337000822753EC0BF030C182F40401300E822717
:1033800053EC0BF031C182F40401300E822753EC70
:103390000BF032C182F40401300E822753EC0BF0A3
:1033A00033C182F40401300E822753EC0BF0040188
:1033B0002C0E826F53EC0BF00101036B026B50C5B6
:1033C00001F14FC500F101AFEBEF19F00101FF0E64
:1033D000026FFF0E036FE9EC2AF02967F2EF19F094
:1033E000F7EF19F004012D0E826F53EC0BF02FC193
:1033F00082F40401300E822753EC0BF030C182F4CA
:103400000401300E822753EC0BF031C182F4040129
:10341000300E822753EC0BF032C182F40401300EDF
:10342000822753EC0BF033C182F40401300E822763
:1034300053EC0BF004012C0E826F53EC0BF00101E6
:10344000036B026B52C501F151C500F101AF2EEFC4
:103450001AF00101FF0E026FFF0E036FE9EC2AF074
:10346000296735EF1AF03AEF1AF004012D0E826F3A
:1034700053EC0BF02FC182F40401300E822753EC81
:103480000BF030C182F40401300E822753EC0BF0B4
:1034900031C182F40401300E822753EC0BF032C1AB
:1034A00082F40401300E822753EC0BF033C182F416
:1034B0000401300E822753EC0BF004012C0E826FB6
:1034C00053EC0BF00101036B026B46C501F145C5DE
:1034D00000F101AF71EF1AF00101FF0E026FFF0E54
:1034E000036FE9EC2AF0296778EF1AF07DEF1AF004
:1034F00004012D0E826F53EC0BF02FC182F40401F6
:10350000300E822753EC0BF030C182F40401300EF0
:10351000822753EC0BF031C182F40401300E822774
:1035200053EC0BF032C182F40401300E822753ECCD
:103530000BF033C182F40401300E822753EC0BF000
:103540000794ABEF1BF087EC2BF085C32AF186C301
:103550002BF187C32CF188C32DF189C32EF18AC3C7
:103560002FF18BC330F18CC331F18DC332F18EC397
:1035700033F10101296B94EC2BF00BEC2BF00101E2
:10358000010E046F000E056F000E066F000E076F30
:103590004BEC2AF0100E046F000E056F000E066F44
:1035A000000E076F5CEC2AF000C129F501C12AF575
:1035B00002C12BF503C12CF5A9EC30F004014C0E2F
:1035C000826F53EC0BF00401460E826F53EC0BF04C
:1035D00004012C0E826F53EC0BF025C500F126C5BB
:1035E00001F127C502F128C503F10101100E046F96
:1035F000000E056F000E066F000E076F7CEC2AF0C0
:10360000E9EC2AF02AC182F40401300E822753EC3F
:103610000BF02BC182F40401300E822753EC0BF027
:103620002CC182F40401300E822753EC0BF02DC123
:1036300082F40401300E822753EC0BF02EC182F489
:103640000401300E822753EC0BF02FC182F40401E9
:10365000300E822753EC0BF030C182F40401300E9F
:10366000822753EC0BF031C182F40401300E822723
:1036700053EC0BF032C182F40401300E822753EC7C
:103680000BF033C182F40401300E822753EC0BF0AF
:10369000ABEF1BF00F987FEC31F098EF23F00401B3
:1036A0004C0E826F53EC0BF00401350E826F53EC1D
:1036B0000BF004012C0E826F53EC0BF046EC2BF058
:1036C0000784B5C500F10794E9EC2AF031C182F412
:1036D0000401300E822753EC0BF032C182F4040156
:1036E000300E822753EC0BF033C182F40401300E0C
:1036F000822753EC0BF0ABEF1BF042EC31F046ECC1
:103700002BF033C500F1E9EC2AF004014C0E826F76
:1037100053EC0BF00401360E826F53EC0BF00401F6
:103720002C0E826F53EC0BF031C182F40401300E89
:10373000822753EC0BF032C182F40401300E822751
:1037400053EC0BF033C182F40401300E822753ECAA
:103750000BF0ABEF1BF05DEC0BF098EF23F00401E6
:103760004C0E826F53EC0BF00401500E826F53EC41
:103770000BF004012C0E826F53EC0BF085C32AF181
:1037800086C32BF187C32CF188C32DF189C32EF199
:103790008AC32FF18BC330F18CC331F18DC332F169
:1037A0008EC333F1010194EC2BF00BEC2BF00301F1
:1037B0008451530A0DE0030184514D0A38E004019D
:1037C000780E826F53EC0BF05DEC0BF098EF23F06A
:1037D0000401530E826F53EC0BF0250E0C6E00C1EA
:1037E0000BF0F9EC07F0260E0C6E01C10BF0F9ECB2
:1037F00007F0270E0C6E02C10BF0F9EC07F0280E53
:103800000C6E03C10BF0F9EC07F000C153F501C1D8
:1038100054F502C155F503C156F500C157F501C174
:1038200058F502C159F503C15AF58CEF1CF004019B
:103830004D0E826F53EC0BF0290E0C6E00C10BF095
:10384000F9EC07F000C15BF500C15CF58CEF1CF0F2
:1038500004014C0E826F53EC0BF00401540E826F86
:1038600053EC0BF004012C0E826F53EC0BF084C36D
:103870002AF185C32BF186C32CF187C32DF188C3B0
:103880002EF189C32FF18AC330F18BC331F18DC37F
:1038900032F18EC333F1010194EC2BF00BEC2BF0E1
:1038A0000101000E046F000E056F010E066F000E81
:1038B000076F5CEC2AF0210E0C6E00C10BF0F9ECE6
:1038C00007F0220E0C6E01C10BF0F9EC07F0230E8D
:1038D0000C6E02C10BF0F9EC07F0240E0C6E03C164
:1038E0000BF0F9EC07F000C15DF501C15EF502C116
:1038F0005FF503C160F58CEF1CF004014C0E826F84
:1039000053EC0BF00401490E826F53EC0BF00401F1
:103910002C0E826F53EC0BF0250E10EC08F0E8CF64
:1039200000F1260E10EC08F0E8CF01F1270E10ECA4
:1039300008F0E8CF02F1280E10EC08F0E8CF03F110
:10394000E9EC2AF0CCEC28F00401730E826F53EC02
:103950000BF004012C0E826F53EC0BF046EC2BF0B5
:10396000290E10EC08F0E8CF00F1E9EC2AF0CCECDD
:1039700028F00401730E826F53EC0BF004012C0E3F
:10398000826F53EC0BF057C500F158C501F159C5D2
:1039900002F15AC503F1E9EC2AF0CCEC28F004015D
:1039A000730E826F53EC0BF004012C0E826F53ECFC
:1039B0000BF046EC2BF05CC500F1E9EC2AF0CCEC06
:1039C00028F004016D0E826F53EC0BF004012C0EF5
:1039D000826F53EC0BF05DC500F15EC501F15FC570
:1039E00002F160C503F1B3EC23F004012C0E826FE9
:1039F00053EC0BF05DEC0BF098EF23F083C32AF14E
:103A000084C32BF185C32CF186C32DF187C32EF11E
:103A100088C32FF189C330F18AC331F18BC332F1EE
:103A20008CC333F1010194EC2BF00BEC2BF0160E50
:103A30000C6E00C10BF0F9EC07F0170E0C6E01C113
:103A40000BF0F9EC07F0180E0C6E02C10BF0F9EC5C
:103A500007F0190E0C6E03C10BF0F9EC07F000C172
:103A60008AF101C18BF102C18CF103C18DF100C15A
:103A70008EF101C18FF102C190F103C191F1E0EF2C
:103A80001DF083C32AF184C32BF185C32CF186C3B7
:103A90002DF187C32EF188C32FF189C330F18AC37A
:103AA00031F18BC332F18CC333F1010194EC2BF073
:103AB0000BEC2BF000C18AF101C18BF102C18CF13A
:103AC00003C18DF100C18EF101C18FF102C190F1EE
:103AD00003C191F1E0EF1DF083C32AF184C32BF100
:103AE00085C32CF186C32DF187C32EF188C32FF136
:103AF00089C330F18AC331F18CC332F18DC333F104
:103B0000010194EC2BF00BEC2BF00101000E046F83
:103B1000000E056F010E066F000E076F5CEC2AF0B9
:103B20001A0E0C6E00C10BF0F9EC07F01B0E0C6EB8
:103B300001C10BF0F9EC07F01C0E0C6E02C10BF08A
:103B4000F9EC07F01D0E0C6E03C10BF0F9EC07F059
:103B500000C192F101C193F102C194F103C195F149
:103B6000E0EF1DF083C32AF184C32BF185C32CF150
:103B700086C32DF187C32EF188C32FF189C330F19D
:103B80008AC331F18CC332F18DC333F1010194EC5E
:103B90002BF00BEC2BF00101000E046F000E056FF3
:103BA000010E066F000E076F5CEC2AF000C192F167
:103BB00001C193F102C194F103C195F1E0EF1DF051
:103BC000160E10EC08F0E8CF00F1170E10EC08F01C
:103BD000E8CF01F1180E10EC08F0E8CF02F1190E51
:103BE00010EC08F0E8CF03F1E9EC2AF0CCEC28F077
:103BF0000401730E826F53EC0BF004012C0E826FE4
:103C000053EC0BF08AC100F18BC101F18CC102F1C0
:103C10008DC103F1E9EC2AF0CCEC28F00401730E1D
:103C2000826F53EC0BF004012C0E826F53EC0BF0FF
:103C30001A0E10EC08F0E8CF00F11B0E10EC08F0A3
:103C4000E8CF01F11C0E10EC08F0E8CF02F11D0ED8
:103C500010EC08F0E8CF03F1B3EC23F004012C0ED4
:103C6000826F53EC0BF092C100F193C101F194C14A
:103C700002F195C103F1B3EC23F05DEC0BF098EF8A
:103C800023F00401690E826F53EC0BF004012C0E3B
:103C9000826F53EC0BF00101040E006F000E016FF8
:103CA000000E026F000E036FE9EC2AF02CC182F4C3
:103CB0000401300E822753EC0BF02DC182F4040175
:103CC000300E822753EC0BF02EC182F40401300E2B
:103CD000822753EC0BF02FC182F40401300E8227AF
:103CE00053EC0BF030C182F40401300E822753EC08
:103CF0000BF031C182F40401300E822753EC0BF03B
:103D000032C182F40401300E822753EC0BF033C130
:103D100082F40401300E822753EC0BF004012C0EC8
:103D2000826F53EC0BF001010B0E006F000E016F60
:103D3000000E026F000E036FE9EC2AF02CC182F432
:103D40000401300E822753EC0BF02DC182F40401E4
:103D5000300E822753EC0BF02EC182F40401300E9A
:103D6000822753EC0BF02FC182F40401300E82271E
:103D700053EC0BF030C182F40401300E822753EC77
:103D80000BF031C182F40401300E822753EC0BF0AA
:103D900032C182F40401300E822753EC0BF033C1A0
:103DA00082F40401300E822753EC0BF004012C0E38
:103DB000826F53EC0BF00101270E006F000E016FB4
:103DC000000E026F000E036FE9EC2AF02CC182F4A2
:103DD0000401300E822753EC0BF02DC182F4040154
:103DE000300E822753EC0BF02EC182F40401300E0A
:103DF000822753EC0BF02FC182F40401300E82278E
:103E000053EC0BF030C182F40401300E822753ECE6
:103E10000BF031C182F40401300E822753EC0BF019
:103E200032C182F40401300E822753EC0BF033C10F
:103E300082F40401300E822753EC0BF004012C0EA7
:103E4000826F53EC0BF0200EF86EF76AF66A0401ED
:103E50000900F5CF82F453EC0BF00900F5CF82F4A2
:103E600053EC0BF00900F5CF82F453EC0BF0090092
:103E7000F5CF82F453EC0BF00900F5CF82F453EC4C
:103E80000BF00900F5CF82F453EC0BF00900F5CFED
:103E900082F453EC0BF00900F5CF82F453EC0BF0F5
:103EA0005DEC0BF098EF23F08351630AD8A498EFF0
:103EB00023F08451610AD8A498EF23F085516C0A4D
:103EC000D8A498EF23F08651410A42E08651440A73
:103ED0001BE08651420AD8B4BBEF1FF08651350A69
:103EE000D8B422EF25F08651360AD8B477EF25F002
:103EF0008651370AD8B4E0EF25F08651380AD8B495
:103F00003EEF26F098EF23F00798079A04017A0E07
:103F1000826F53EC0BF00401780E826F53EC0BF0C0
:103F20000401640E826F53EC0BF081A89FEF1FF029
:103F30000401550E826F53EC0BF0A4EF1FF0040147
:103F40004C0E826F53EC0BF05DEC0BF098EF23F00E
:103F50000788079A04017A0E826F53EC0BF0040174
:103F6000410E826F53EC0BF00401610E826F53EC33
:103F70000BF095EF1FF00798078A04017A0E826F05
:103F800053EC0BF00401420E826F53EC0BF0040172
:103F9000610E826F53EC0BF095EF1FF00101666725
:103FA000D9EF1FF06767D9EF1FF06867D9EF1FF0EF
:103FB0006967F1EF1FF04F67E5EF1FF05067E5EF1E
:103FC0001FF05167E5EF1FF05267F1EF1FF001019D
:103FD000000E006F000E016F000E026F000E036FE7
:103FE00012000101620E046F010E056F000E066FD4
:103FF000000E076F66C100F167C101F168C102F1EF
:1040000069C103F14BEC2AF003BF75EF20F0010109
:10401000000E046FA80E056F550E066F020E076F97
:1040200066C100F167C101F168C102F169C103F124
:1040300066C186F167C187F168C188F169C189F1FC
:104040004BEC2AF003BF2EEF20F00101000E866F2B
:10405000A80E876F550E886F020E896F0E0E10EC3A
:1040600008F0E8CF18F10F0E10EC08F0E8CF19F1C6
:10407000100E10EC08F0E8CF1AF1110E10EC08F059
:10408000E8CF1BF194EC29F086C104F187C105F15A
:1040900088C106F189C107F14BEC2AF0078258EC80
:1040A00029F094EC29F0079258EC29F086C100F130
:1040B00087C101F188C102F189C103F1079258EC6F
:1040C00029F0CC0E046FE00E056F870E066F050E0B
:1040D000076F4BEC2AF000C118F101C119F102C1C0
:1040E0001AF103C11BF1ADEF20F00101800E006F4A
:1040F0001A0E016F060E026F000E036F4FC104F11E
:1041000050C105F151C106F152C107F14BEC2AF043
:1041100003AF8EEF20F046EC2BF012000E0E10ECE9
:1041200008F0E8CF18F10F0E10EC08F0E8CF19F105
:10413000100E10EC08F0E8CF1AF1110E10EC08F098
:10414000E8CF1BF14FC100F150C101F151C102F1A3
:1041500052C103F1078258EC29F018C100F119C1CE
:1041600001F11AC102F11BC103F112000401730E27
:10417000826F53EC0BF004012C0E826F53EC0BF0AA
:10418000078462C166F163C167F164C168F165C10A
:1041900069F14BC14FF14CC150F14DC151F14EC1CC
:1041A00052F157C159F158C15AF10794DCEC20F093
:1041B0005DEC0BF098EF23F066C100F167C101F1EF
:1041C00068C102F169C103F10101E9EC2AF0CCEC0C
:1041D00028F00401630E826F53EC0BF004012C0EE7
:1041E000826F53EC0BF04FC100F150C101F151C18E
:1041F00002F152C103F10101E9EC2AF0CCEC28F004
:104200000401660E826F53EC0BF004012C0E826FDA
:1042100053EC0BF046EC2BF059C100F15AC101F1FF
:104220000101E9EC2AF0CCEC28F00401740E826F55
:1042300053EC0BF0120010820401530E826F53EC0A
:104240000BF004012C0E826F53EC0BF083C32AF1A8
:1042500084C32BF185C32CF186C32DF187C32EF1C6
:1042600088C32FF189C330F18AC331F18BC332F196
:104270008CC333F1010194EC2BF00BEC2BF000C15B
:1042800066F101C167F102C168F103C169F18EC332
:104290002AF18FC32BF190C32CF191C32DF192C35E
:1042A0002EF193C32FF194C330F195C331F196C32E
:1042B00032F197C333F1010194EC2BF00BEC2BF0AE
:1042C00000C14FF101C150F102C151F103C152F1DE
:1042D00087EC2BF099C32FF19AC330F19BC331F1D6
:1042E0009CC332F19DC333F1010194EC2BF00BEC34
:1042F0002BF000C159F101C15AF1DCEC20F00401AE
:104300002C0E826F53EC0BF08DEF21F08251520A8C
:1043100003E10F828DEF21F00F928251750A03E1C4
:10432000108494EF21F010948251550A03E1108615
:104330009BEF21F01096078410B2F8EF21F010A443
:10434000E4EF21F0B6C166F1B7C167F1B8C168F119
:10435000B9C169F1BAC16AF1BBC16BF1BCC16CF101
:10436000BDC16DF1BEC16EF1BFC16FF1C0C170F1D1
:10437000C1C171F1C2C172F1C3C173F1C4C174F1A1
:10438000C5C175F1C6C176F1C7C177F1C8C178F171
:10439000C9C179F1CAC17AF1CBC17BF1CCC17CF141
:1043A000CDC17DF1CEC17EF1CFC17FF1D0C180F111
:1043B000D1C181F1D2C182F1D3C183F1D4C184F1E1
:1043C000D5C185F1ECEF21F062C166F163C167F1FF
:1043D00064C168F165C169F14BC14FF14CC150F145
:1043E0004DC151F14EC152F157C159F158C15AF165
:1043F00007940FA01AEF22F00101926707EF22F055
:10440000936707EF22F0946707EF22F095670BEFB1
:1044100022F01AEF22F0CEEC1FF092C104F193C10A
:1044200005F194C106F195C107F14BEC2AF003BFE9
:104430005EEF23F0CEEC1FF00101000E046F000EC2
:10444000056F010E066F000E076F7CEC2AF010A4BA
:1044500031EF22F00401750E826F53EC0BF036EF52
:1044600022F00401720E826F53EC0BF004012C0E4B
:10447000826F53EC0BF0E9EC2AF0296745EF22F04C
:104480000401200E826F48EF22F004012D0E826F8E
:1044900053EC0BF030C182F40401300E822753EC50
:1044A0000BF031C182F40401300E822753EC0BF083
:1044B00004012E0E826F53EC0BF032C182F4040122
:1044C000300E822753EC0BF033C182F40401300E1E
:1044D000822753EC0BF004016D0E826F53EC0BF04E
:1044E00004012C0E826F53EC0BF04FC100F150C150
:1044F00001F151C102F152C103F10101E9EC2AF0CD
:10450000CCEC28F00401480E826F53EC0BF0040150
:104510007A0E826F53EC0BF004012C0E826F53EC79
:104520000BF066C100F167C101F168C102F169C118
:1045300003F10101E9EC2AF0CCEC28F00401630E50
:10454000826F53EC0BF004012C0E826F53EC0BF0D6
:1045500066C100F167C101F168C102F169C103F1EF
:1045600001010A0E046F000E056F000E066F000EAB
:10457000076F5CEC2AF0000E046F120E056F000E40
:10458000066F000E076F7CEC2AF0E9EC2AF02AC1D6
:1045900082F40401300E822753EC0BF02BC182F41D
:1045A0000401300E822753EC0BF02CC182F404017D
:1045B000300E822753EC0BF02DC182F40401300E33
:1045C000822753EC0BF02EC182F40401300E8227B7
:1045D00053EC0BF02FC182F40401300E822753EC10
:1045E0000BF030C182F40401300E822753EC0BF043
:1045F00004012E0E826F53EC0BF031C182F40401E2
:10460000300E822753EC0BF032C182F40401300EDD
:10461000822753EC0BF033C182F40401300E822761
:1046200053EC0BF00401730E826F53EC0BF004019A
:104630002C0E826F53EC0BF046EC2BF059C100F1BD
:104640005AC101F1C2EC24F00FB22AEF23F00FA0FF
:104650005CEF23F004012C0E826F53EC0BF0200E64
:10466000F86EF76AF66A04010900F5CF82F453EC9C
:104670000BF00900F5CF82F453EC0BF00900F5CFF5
:1046800082F453EC0BF00900F5CF82F453EC0BF0FD
:104690000900F5CF82F453EC0BF00900F5CF82F45A
:1046A00053EC0BF00900F5CF82F453EC0BF009004A
:1046B000F5CF82F453EC0BF05DEC0BF00F9098EF1C
:1046C00023F00401630E826F53EC0BF004012C0EF7
:1046D000826F53EC0BF09EEC23F004012C0E826FE2
:1046E00053EC0BF011EC24F004012C0E826F53EC10
:1046F0000BF08DEC24F004012C0E826F53EC0BF0C8
:104700000101F80E006FCD0E016F660E026F030EF1
:10471000036FB3EC23F004012C0E826F53EC0BF00B
:10472000A3EC24F05DEC0BF098EF23F05DEC0BF0C4
:104730000301C26B07901092A7EF26F0D8900E0EDF
:1047400010EC08F0E8CF00F10F0E10EC08F0E8CF05
:1047500001F1100E10EC08F0E8CF02F1110E10EC90
:1047600008F0E8CF03F10101000E046F000E056FA1
:10477000010E066F000E076F7CEC2AF0E9EC2AF0C0
:104780002AC182F40401300E822753EC0BF02BC1B6
:1047900082F40401300E822753EC0BF02CC182F41A
:1047A0000401300E822753EC0BF02DC182F404017A
:1047B000300E822753EC0BF02EC182F40401300E30
:1047C000822753EC0BF02FC182F40401300E8227B4
:1047D00053EC0BF030C182F40401300E822753EC0D
:1047E0000BF031C182F40401300E822753EC0BF040
:1047F00004012E0E826F53EC0BF032C182F40401DF
:10480000300E822753EC0BF033C182F40401300EDA
:10481000822753EC0BF004016D0E826F53EC0BF00A
:104820001200120E10EC08F0E8CF00F1130E10EC9D
:1048300008F0E8CF01F1140E10EC08F0E8CF02F117
:10484000150E10EC08F0E8CF03F101010A0E046F19
:10485000000E056F000E066F000E076F5CEC2AF06D
:10486000000E046F120E056F000E066F000E076F2C
:104870007CEC2AF0E9EC2AF02AC182F40401300E23
:10488000822753EC0BF02BC182F40401300E8227F7
:1048900053EC0BF02CC182F40401300E822753EC50
:1048A0000BF02DC182F40401300E822753EC0BF083
:1048B0002EC182F40401300E822753EC0BF02FC17D
:1048C00082F40401300E822753EC0BF030C182F4E5
:1048D0000401300E822753EC0BF004012E0E826F80
:1048E00053EC0BF031C182F40401300E822753ECFB
:1048F0000BF032C182F40401300E822753EC0BF02E
:1049000033C182F40401300E822753EC0BF0040112
:10491000730E826F53EC0BF012000A0E10EC08F0CD
:10492000E8CF00F10B0E10EC08F0E8CF01F10C0E0F
:1049300010EC08F0E8CF02F10D0E10EC08F0E8CF13
:1049400003F1C2EF24F0060E10EC08F0E8CF00F1FE
:10495000070E10EC08F0E8CF01F1080E10EC08F09B
:10496000E8CF02F1090E10EC08F0E8CF03F1C2EF36
:1049700024F0010146EC2BF0078457C100F158C127
:1049800001F107940101E80E046F800E056F000E1F
:10499000066F000E076F5CEC2AF0000E046F040E29
:1049A000056F000E066F000E076F7CEC2AF0880E74
:1049B000046F130E056F000E066F000E076F4BECB1
:1049C0002AF00A0E046F000E056F000E066F000E2F
:1049D000076F7CEC2AF0E9EC2AF001012967F6EF79
:1049E00024F00401200E826FF9EF24F004012D0E53
:1049F000826F53EC0BF030C182F40401300E822739
:104A000053EC0BF031C182F40401300E822753ECD9
:104A10000BF032C182F40401300E822753EC0BF00C
:104A200004012E0E826F53EC0BF033C182F40401AB
:104A3000300E822753EC0BF00401430E826F53ECCF
:104A40000BF0120087C32AF188C32BF189C32CF124
:104A50008AC32DF18BC32EF18CC32FF18DC330F19E
:104A60008EC331F190C332F191C333F10101296B4F
:104A700094EC2BF00BEC2BF00101000E046F000EF8
:104A8000056F010E066F000E076F5CEC2AF00E0E2C
:104A90000C6E00C10BF0F9EC07F00F0E0C6E01C1AB
:104AA0000BF0F9EC07F0100E0C6E02C10BF0F9ECF4
:104AB00007F0110E0C6E03C10BF0F9EC07F00401C6
:104AC0007A0E826F53EC0BF004012C0E826F53ECC4
:104AD0000BF00401350E826F53EC0BF004012C0E29
:104AE000826F53EC0BF09EEC23F0A4EF1FF087C312
:104AF0002AF188C32BF189C32CF18AC32DF18BC312
:104B00002EF18CC32FF18DC330F18EC331F190C3E0
:104B100032F191C333F10101296B94EC2BF00BECD2
:104B20002BF0880E046F130E056F000E066F000E3B
:104B3000076F50EC2AF0000E046F040E056F000E94
:104B4000066F000E076F5CEC2AF00101E80E046F9F
:104B5000800E056F000E066F000E076F7CEC2AF0CA
:104B60000A0E0C6E00C10BF0F9EC07F00B0E0C6E88
:104B700001C10BF0F9EC07F00C0E0C6E02C10BF04A
:104B8000F9EC07F00D0E0C6E03C10BF0F9EC07F019
:104B900004017A0E826F53EC0BF004012C0E826F2D
:104BA00053EC0BF00401360E826F53EC0BF0040152
:104BB0002C0E826F53EC0BF08DEC24F0A4EF1FF061
:104BC00087C32AF188C32BF189C32CF18AC32DF145
:104BD0008BC32EF18CC32FF18DC330F18FC331F114
:104BE00090C332F191C333F1010194EC2BF00BEC43
:104BF0002BF0000E046F120E056F000E066F000EF4
:104C0000076F5CEC2AF001010A0E046F000E056FBD
:104C1000000E066F000E076F7CEC2AF0120E0C6E71
:104C200000C10BF0F9EC07F0130E0C6E01C10BF094
:104C3000F9EC07F0140E0C6E02C10BF0F9EC07F062
:104C4000150E0C6E03C10BF0F9EC07F004017A0E9F
:104C5000826F53EC0BF004012C0E826F53EC0BF0BF
:104C60000401370E826F53EC0BF004012C0E826F9F
:104C700053EC0BF011EC24F0A4EF1FF087C32AF1E2
:104C800088C32BF189C32CF18AC32DF18BC32EF17C
:104C90008CC32FF18DC330F18EC331F190C332F14B
:104CA00091C333F10101296B94EC2BF00BEC2BF049
:104CB000880E046F130E056F000E066F000E076F4F
:104CC00050EC2AF0000E046F040E056F000E066F04
:104CD000000E076F5CEC2AF00101E80E046F800EF5
:104CE000056F000E066F000E076F7CEC2AF0060EB3
:104CF0000C6E00C10BF0F9EC07F0070E0C6E01C151
:104D00000BF0F9EC07F0080E0C6E02C10BF0F9EC99
:104D100007F0090E0C6E03C10BF0F9EC07F004016B
:104D20007A0E826F53EC0BF004012C0E826F53EC61
:104D30000BF00401380E826F53EC0BF004012C0EC3
:104D4000826F53EC0BF0A3EC24F0A4EF1FF081A8CA
:104D500065EF27F007A81EEF27F00101800E006F16
:104D60001A0E016F060E026F000E036F4BC104F1A5
:104D70004CC105F14DC106F14EC107F14BEC2AF0D3
:104D800003BF65EF27F0C6EC28F04BC100F14CC122
:104D900001F14DC102F14EC103F1078258EC29F037
:104DA00018C104F119C105F11AC106F11BC107F1BF
:104DB000F80E006FCD0E016F660E026F030E036FCB
:104DC0004BEC2AF00E0E0C6E00C10BF0F9EC07F064
:104DD0000F0E0C6E01C10BF0F9EC07F0100E0C6E0B
:104DE00002C10BF0F9EC07F0110E0C6E03C10BF0D1
:104DF000F9EC07F00784010146EC2BF057C100F1F4
:104E000058C101F107940A0E0C6E00C10BF0F9ECC9
:104E100007F00B0E0C6E01C10BF0F9EC07F00C0E55
:104E20000C6E02C10BF0F9EC07F00D0E0C6E03C115
:104E30000BF0F9EC07F0079865EF27F007AA65EF8C
:104E400027F00784010146EC2BF057C100F158C14F
:104E500001F10794060E0C6E00C10BF0F9EC07F09F
:104E6000070E0C6E01C10BF0F9EC07F0080E0C6E8A
:104E700002C10BF0F9EC07F0090E0C6E03C10BF048
:104E8000F9EC07F0078462C100F163C101F164C16C
:104E900002F165C103F10794120E0C6E00C10BF014
:104EA000F9EC07F0130E0C6E01C10BF0F9EC07F0F2
:104EB000140E0C6E02C10BF0F9EC07F0150E0C6E1F
:104EC00003C10BF0F9EC07F0079A04018051811936
:104ED0007F0B0BE09EA809D014EE00F081517F0BF0
:104EE000E126E750812B0F01AD6E05012F51010A1C
:104EF00013E081AA8CEF27F005012F51000A0AE088
:104F00000FB88CEF27F0050130678CEF27F00FB852
:104F10008CEF27F003EF35F081B8A1EF27F095EC87
:104F20002DF005012F51020A02E0A1EF27F05C2FBE
:104F3000A1EF27F05BC55CF50501010E306F3C0E5B
:104F4000316FB2EF0AF006013251385D3351D8A00B
:104F5000010F395D800BD8A4B2EF27F032C638F6C6
:104F600033C639F6120006013251365D3351D8A0EE
:104F7000010F375D800BD8B4C2EF27F032C636F68A
:104F800033C637F6120007841AC632F61BC633F64C
:104F90001CC638F61DC639F6A3EC27F01EC632F63D
:104FA0001FC633F6A3EC27F020C632F621C633F62F
:104FB000A3EC27F01AC632F61BC633F61CC636F62B
:104FC0001DC637F6B3EC27F01EC632F61FC633F601
:104FD000B3EC27F020C632F621C633F6B3EC27F047
:104FE0003851365F3951D8A03929375F46EC2BF05C
:104FF00036C600F137C601F152EC2BF000C13AF68B
:1050000001C13BF622C632F623C633F624C638F673
:1050100025C639F6A3EC27F026C632F627C633F6A6
:10502000A3EC27F028C632F629C633F6A3EC27F006
:1050300022C632F623C633F624C636F625C637F620
:10504000B3EC27F026C632F627C633F6B3EC27F0CA
:1050500028C632F629C633F6B3EC27F03851365F4E
:105060003951D8A03929375F46EC2BF036C600F10C
:1050700037C601F152EC2BF000C13CF601C13DF600
:105080002AC632F62BC633F62CC638F62DC639F6AC
:10509000A3EC27F02EC632F62FC633F6A3EC27F08A
:1050A00030C632F631C633F6A3EC27F02AC632F604
:1050B0002BC633F62CC636F62DC637F6B3EC27F0E2
:1050C0002EC632F62FC633F6B3EC27F030C632F6D2
:1050D00031C633F6B3EC27F03851365F3951D8A0DA
:1050E0003929375F46EC2BF036C600F137C601F19F
:1050F00052EC2BF000C13EF601C13FF63AC632F643
:105100003BC633F63CC636F63DC637F6B3EC27F061
:105110003EC632F63FC633F6B3EC27F007941200D2
:1051200018C100F119C101F11AC102F11BC103F14B
:10513000000E046F000E056F010E066F000E076F64
:105140007CEC2AF029A1BBEF28F02051D8B4BBEFAA
:1051500028F018C100F119C101F11AC102F11BC1F7
:1051600003F1000E046F000E056F0A0E066F000EAD
:10517000076F7CEC2AF01200010104510013055165
:105180000113065102130751031312000101186B9A
:10519000196B1A6B1B6B12002AC182F40401300ECA
:1051A000822753EC0BF02BC182F40401300E8227CE
:1051B00053EC0BF02CC182F40401300E822753EC27
:1051C0000BF02DC182F40401300E822753EC0BF05A
:1051D0002EC182F40401300E822753EC0BF02FC154
:1051E00082F40401300E822753EC0BF030C182F4BC
:1051F0000401300E822753EC0BF031C182F404011C
:10520000300E822753EC0BF032C182F40401300ED1
:10521000822753EC0BF033C182F40401300E822755
:1052200053EC0BF012002FC182F40401300E8227E0
:1052300053EC0BF030C182F40401300E822753ECA2
:105240000BF031C182F40401300E822753EC0BF0D5
:1052500032C182F40401300E822753EC0BF033C1CB
:1052600082F40401300E822753EC0BF01200060E7C
:10527000116E060E126E060E136E112E3DEF29F002
:10528000122E3DEF29F0132E3DEF29F08B84020EF4
:10529000116E020E126E020E136E112E4DEF29F0DA
:1052A000122E4DEF29F0132E4DEF29F08B941200A2
:1052B0000101005305E1015303E1025301E1002B19
:1052C0001BEC2AF046EC2BF03951006F3A51016F7C
:1052D000420E046F4B0E056F000E066F000E076F37
:1052E0005CEC2AF000C104F101C105F102C106F134
:1052F00003C107F118C100F119C101F11AC102F18E
:105300001BC103F107B289EF29F050EC2AF08BEFB3
:1053100029F04BEC2AF000C118F101C119F102C1CA
:105320001AF103C11BF1120046EC2BF059C100F138
:105330005AC101F1060E10EC08F0E8CF04F1070E97
:1053400010EC08F0E8CF05F1080E10EC08F0E8CFFB
:1053500006F1090E10EC08F0E8CF07F14BEC2AF04B
:1053600000C124F101C125F102C126F103C127F1D9
:10537000290E046F000E056F000E066F000E076FFA
:105380005CEC2AF0EE0E046F430E056F000E066F04
:10539000000E076F50EC2AF024C104F125C105F17D
:1053A00026C106F127C107F15CEC2AF000C11CF10F
:1053B00001C11DF102C11EF103C11FF1120E10EC5B
:1053C00008F0E8CF04F1130E10EC08F0E8CF05F177
:1053D000140E10EC08F0E8CF06F1150E10EC08F0F2
:1053E000E8CF07F10D0E006F000E016F000E026F87
:1053F000000E036F5CEC2AF0180E046F000E056FB0
:10540000000E066F000E076F7CEC2AF01CC104F141
:105410001DC105F11EC106F11FC107F150EC2AF0B4
:105420006A0E046F2A0E056F000E066F000E076FDE
:105430004BEC2AF01200BF0EFA6E200E3A6F396B59
:10544000D8900037013702370337D8B02CEF2AF055
:105450003A2F21EF2AF039073A070353D8B4120044
:105460000331070B80093F6F03390F0B010F396FB1
:1054700080EC5FF0406F390580EC5FF0405D405F8D
:10548000396B3F33D8B0392739333FA941EF2AF080
:1054900040513927120001016BEC2BF0D8B01200FB
:1054A000010103510719346F2EEC2BF0D8900751EE
:1054B000031934AF800F12000101346B52EC2BF052
:1054C000D8A068EC2BF0D8B012003DEC2BF046ECE5
:1054D0002BF01F0E366F7EEC2BF00B35D8B02EEC78
:1054E0002BF0D8A00335D8B01200362F6BEF2AF07E
:1054F00034B155EC2BF012000101346B045105114D
:10550000061107110008D8A052EC2BF0D8A068ECC7
:105510002BF0D8B01200086B096B0A6B0B6B7EEC9A
:105520002BF01F0E366F7EEC2BF007510B5DD8A4CD
:10553000A6EF2AF006510A5DD8A4A6EF2AF005517D
:10554000095DD8A4A6EF2AF00451085DD8A0B9EFF0
:105550002AF00451085F0551D8A0053D095F0651A6
:10556000D8A0063D0A5F0751D8A0073D0B5FD89031
:105570000081362F93EF2AF034B155EC2BF0346BC9
:1055800052EC2BF0D89082EC2BF007510B5DD8A495
:10559000D6EF2AF006510A5DD8A4D6EF2AF00551BD
:1055A000095DD8A4D6EF2AF00451085DD8A0E5EF34
:1055B0002AF0003FE5EF2AF0013FE5EF2AF0023F35
:1055C000E5EF2AF0032BD8B4120034B155EC2BF0E0
:1055D00012000101346B52EC2BF0D8B0120087ECB2
:1055E0002BF0200E366F003701370237033711EEEC
:1055F00033F00A0E376FE7360A0EE75CD8B0E76E75
:10560000E552372FFBEF2AF0362FF3EF2AF034B1B3
:105610002981D890120001010A0E346F200E366FD6
:1056200011EE29F03451376F0A0ED890E652D8B0F7
:10563000E726E732372F16EF2BF00333023301331F
:105640000033362F10EF2BF0E750FF0FD8A00335B3
:10565000D8B0120029B155EC2BF0120004510027EC
:105660000551D8B0053D01270651D8B0063D0227A7
:105670000751D8B0073D032712000051086F0151B0
:10568000096F02510A6F03510B6F12000101006B89
:10569000016B026B036B12000101046B056B066B5F
:1056A000076B12000335D8A012000351800B001FB6
:1056B000011F021F031F003F65EF2BF0013F65EF45
:1056C0002BF0023F65EF2BF0032B342B0325120048
:1056D0000735D8A012000751800B041F051F061FB5
:1056E000071F043F7BEF2BF0053F7BEF2BF0063FBE
:1056F0007BEF2BF0072B342B0725120000370137E7
:1057000002370337083709370A370B371200010110
:10571000296B2A6B2B6B2C6B2D6B2E6B2F6B306BCD
:10572000316B326B336B120001012A510F0B2A6F60
:105730002B510F0B2B6F2C510F0B2C6F2D510F0B6F
:105740002D6F2E510F0B2E6F2F510F0B2F6F3051CE
:105750000F0B306F31510F0B316F32510F0B326F16
:1057600033510F0B336F1200899C000EC76E200E51
:10577000C66E9E96C69EC50EC96EFF0E9EB602D020
:10578000E82EFCD79E96C69E000EC96EFF0E9EB6F2
:1057900002D0E82EFCD7C9CF00F69E96C69E000E1A
:1057A000C96EFF0E9EB602D0E82EFCD7C9CF01F617
:1057B000898C1200000EC76E200EC66E899C9E96C4
:1057C000C69EC80EC96EFF0E9EB602D0E82EFCD74C
:1057D0009E96C69E000EC96EFF0E9EB602D0E82EA3
:1057E000FCD7C9CF02F69E96C69E000EC96EFF0E6C
:1057F0009EB602D0E82EFCD7C9CF03F69E96C69E71
:10580000000EC96EFF0E9EB602D0E82EFCD7C9CF9F
:105810000AF69E96C69E000EC96EFF0E9EB602D078
:10582000E82EFCD7C9CF0BF69E96C69E000EC96E19
:10583000FF0E9EB602D0E82EFCD7C9CF12F69E9678
:10584000C69E000EC96EFF0E9EB602D0E82EFCD793
:10585000C9CF13F6898C1200000EC76E200EC66EDB
:10586000899C9E96C69EE80EC96EFF0E9EB602D01B
:10587000E82EFCD79E96C69E000EC96EFF0E9EB601
:1058800002D0E82EFCD7C9CF1AF69E96C69E000E0F
:10589000C96EFF0E9EB602D0E82EFCD7C9CF1BF60C
:1058A0009E96C69E000EC96EFF0E9EB602D0E82ED2
:1058B000FCD7C9CF22F69E96C69E000EC96EFF0E7B
:1058C0009EB602D0E82EFCD7C9CF23F69E96C69E80
:1058D000000EC96EFF0E9EB602D0E82EFCD7C9CFCF
:1058E0002AF69E96C69E000EC96EFF0E9EB602D088
:1058F000E82EFCD7C9CF2BF6898C1200000EC76E9C
:10590000200EC66E899C9E96C69E240EC96EFF0E02
:105910009EB602D0E82EFCD79E96C69EE40EC96EB7
:10592000FF0E9EB602D0E82EFCD7898C899C9E96ED
:10593000C69E200EC96EFF0E9EB602D0E82EFCD782
:105940009E96C69E5F0EC96EFF0E9EB602D0E82ED2
:10595000FCD7898C899C9E96C69E210EC96EFF0E2F
:105960009EB602D0E82EFCD79E96C69EC00EC96E8B
:10597000FF0E9EB602D0E82EFCD7898C899C9E969D
:10598000C69E260EC96EFF0E9EB602D0E82EFCD72C
:105990009E96C69E000EC96EFF0E9EB602D0E82EE1
:1059A000FCD7898C120010A806D08994000EC76E0F
:1059B000220EC66E05D08984000EC76E220EC66EFA
:1059C000050EE82EFED7120010A802D0898401D05F
:1059D0008994050EE82EFED71200D3EC2CF09E968B
:1059E000C69E000EC96EFF0E9EB602D0E82EFCD7F2
:1059F0009E96C69E000EC96EFF0E9EB602D0E82E81
:105A0000FCD7C9CFABF59E96C69E000EC96EFF0EA1
:105A10009EB602D0E82EFCD7C9CFACF59E96C69EA6
:105A2000000EC96EFF0E9EB602D0E82EFCD7C9CF7D
:105A3000ADF59E96C69E000EC96EFF0E9EB602D0B4
:105A4000E82EFCD7C9CFAEF59E96C69E000EC96E55
:105A5000FF0E9EB602D0E82EFCD7C9CFAFF59E96BA
:105A6000C69E000EC96EFF0E9EB602D0E82EFCD771
:105A7000C9CFB0F59E96C69E000EC96EFF0E9EB6AB
:105A800002D0E82EFCD7C9CFB1F5E4EC2CF012001F
:105A9000D3EC2CF09E96C69E800EC96EFF0E9EB66D
:105AA00002D0E82EFCD79E96C69EABC5C9FFFF0E5E
:105AB0009EB602D0E82EFCD79E96C69EACC5C9FF06
:105AC000FF0E9EB602D0E82EFCD79E96C69EADC5B0
:105AD000C9FFFF0E9EB602D0E82EFCD79E96C69E4A
:105AE000AEC5C9FFFF0E9EB602D0E82EFCD79E962B
:105AF000C69EAFC5C9FFFF0E9EB602D0E82EFCD7EA
:105B00009E96C69EB0C5C9FFFF0E9EB602D0E82E77
:105B1000FCD79E96C69EB1C5C9FFFF0E9EB602D0A9
:105B2000E82EFCD7E4EC2CF01200D3EC2CF09E967F
:105B3000C69E070EC96EFF0E9EB602D0E82EFCD799
:105B40009E96C69E000EC96EFF0E9EB602D0E82E2F
:105B5000FCD7C9CFABF59E96C69E000EC96EFF0E50
:105B60009EB602D0E82EFCD7C9CFACF59E96C69E55
:105B7000000EC96EFF0E9EB602D0E82EFCD7C9CF2C
:105B8000ADF59E96C69E000EC96EFF0E9EB602D063
:105B9000E82EFCD7C9CFAEF5E4EC2CF0D3EC2CF01A
:105BA0009E96C69E15C0C9FFFF0E9EB602D0E82E77
:105BB000FCD79E96C69E000EC96EFF0E9EB602D002
:105BC000E82EFCD7C9CFB2F5E4EC2CF01200D3ECF0
:105BD0002CF09E96C69E870EC96EFF0E9EB602D012
:105BE000E82EFCD79E96C69EABC5C9FFFF0E9EB69B
:105BF00002D0E82EFCD79E96C69EACC5C9FFFF0E0C
:105C00009EB602D0E82EFCD79E96C69EADC5C9FFB3
:105C1000FF0E9EB602D0E82EFCD79E96C69EAEC55D
:105C2000C9FFFF0E9EB602D0E82EFCD7E4EC2CF0A4
:105C3000D3EC2CF09E96C69E16C0C9FFFF0E9EB6F2
:105C400002D0E82EFCD79E96C69EB2C5C9FFFF0EB5
:105C50009EB602D0E82EFCD7E4EC2CF01200D3EC78
:105C60002CF09E96C69E870EC96EFF0E9EB602D081
:105C7000E82EFCD79E96C69E000EC96EFF0E9EB6FD
:105C800002D0E82EFCD79E96C69E800EC96EFF0EEF
:105C90009EB602D0E82EFCD79E96C69E800EC96E98
:105CA000FF0E9EB602D0E82EFCD79E96C69E800EB2
:105CB000C96EFF0E9EB602D0E82EFCD7E4EC2CF0A5
:105CC0001200D3EC2CF09E96C69E870EC96EFF0E76
:105CD0009EB602D0E82EFCD79E96C69E000EC96ED8
:105CE000FF0E9EB602D0E82EFCD79E96C69E000EF2
:105CF000C96EFF0E9EB602D0E82EFCD79E96C69EB9
:105D0000800EC96EFF0E9EB602D0E82EFCD79E967E
:105D1000C69E800EC96EFF0E9EB602D0E82EFCD73E
:105D2000E4EC2CF0120010A82DD0D3EC2CF09E96B1
:105D3000C69E16C0C9FFFF0E9EB602D0E82EFCD745
:105D40009E96C69E450EC96EFF0E9EB602D0E82EE8
:105D5000FCD7E4EC2CF0D3EC2CF09E96C69E8F0E74
:105D6000C96EFF0E9EB602D0E82EFCD79E96C69E48
:105D7000000EC96EFF0E9EB602D0E82EFCD7E4ECF2
:105D80002CF01200D3EC2CF09E96C69E16C0C9FFD4
:105D9000FF0E9EB602D0E82EFCD79E96C69E010E40
:105DA000C96EFF0E9EB602D0E82EFCD7E4EC2CF0B4
:105DB000D3EC2CF09E96C69E910EC96EFF0E9EB639
:105DC00002D0E82EFCD79E96C69EA50EC96EFF0E89
:105DD0009EB602D0E82EFCD7E4EC2CF01200D3ECF7
:105DE0002CF09E96C69E16C0C9FFFF0E9EB602D02E
:105DF000E82EFCD79E96C69E810EC96EFF0E9EB6FB
:105E000002D0E82EFCD7E4EC2CF01200D3EC2CF0FE
:105E10009E96C69E16C0C9FFFF0E9EB602D0E82E03
:105E2000FCD79E96C69E010EC96EFF0E9EB602D08E
:105E3000E82EFCD7E4EC2CF01200D3EC2CF09E966C
:105E4000C69E910EC96EFF0E9EB602D0E82EFCD7FC
:105E50009E96C69EA50EC96EFF0E9EB602D0E82E77
:105E6000FCD7E4EC2CF01200D3EC2CF09E96C69EEE
:105E7000910EC96EFF0E9EB602D0E82EFCD79E96FC
:105E8000C69E000EC96EFF0E9EB602D0E82EFCD74D
:105E9000E4EC2CF012000501256B266B276B286BB8
:105EA000899A400EC76E200EC66E9E96C69E030E41
:105EB000C96EFF0E9EB602D0E82EFCD79E96C69EF7
:105EC00027C5C9FFFF0E9EB602D0E82EFCD79E96CE
:105ED000C69E26C5C9FFFF0E9EB602D0E82EFCD78F
:105EE0009E96C69E25C5C9FFFF0E9EB602D0E82E1F
:105EF000FCD79E96C69EC952FF0E9EB602D0E82ED3
:105F0000FCD7898A0F01C950FF0A01E1120005017F
:105F10002E51130A05E005012E51170A0CE012005C
:105F20000501E00E256FFF0E266F0F0E276F000E86
:105F3000286FA4EF2FF00501E00E256FFF0E266FEE
:105F4000FF0E276F000E286F899A400EC76E200E35
:105F5000C66E9E96C69E030EC96EFF0E9EB602D0FA
:105F6000E82EFCD79E96C69E27C5C9FFFF0E9EB69B
:105F700002D0E82EFCD79E96C69E26C5C9FFFF0E0E
:105F80009EB602D0E82EFCD79E96C69E25C5C9FFB8
:105F9000FF0E9EB602D0E82EFCD79E96C69EC95232
:105FA000FF0E9EB602D0E82EFCD7898A0F01C95099
:105FB000FF0A1DE005012E51130A05E005012E51CF
:105FC000170A0BE012000501000E256F000E266F68
:105FD000100E276F000E286F12000501000E256FAE
:105FE000000E266F000E276F010E286F12000501AC
:105FF000256B266B276B286B05012E51130A05E0D4
:1060000005012E51170A0CE012000501000E216F48
:10601000000E226F080E236F000E246F19EF30F070
:106020000501000E216F000E226F800E236F000EFF
:10603000246F21C500F122C501F123C502F124C559
:1060400003F125C504F126C505F127C506F128C5CC
:1060500007F1BCEC28F000C125F501C126F502C10D
:1060600027F503C128F5899A400EC76E200EC66E2B
:106070009E96C69E030EC96EFF0E9EB602D0E82EF7
:10608000FCD79E96C69E27C5C9FFFF0E9EB602D0BE
:10609000E82EFCD79E96C69E26C5C9FFFF0E9EB66B
:1060A00002D0E82EFCD79E96C69E25C5C9FFFF0EDE
:1060B0009EB602D0E82EFCD79E96C69EC952FF0E11
:1060C0009EB602D0E82EFCD7898AC950FF0A08E1A3
:1060D00004C125F505C126F506C127F507C128F538
:1060E000D890050124332333223321332151E00B8F
:1060F000216F216783EF30F0226783EF30F0236751
:1061000083EF30F0246719EF30F00501200E2527CA
:10611000E86A2623E86A2723E86A28231200E86A47
:1061200005012E51130A06E005012E51170A0BE056
:10613000020E120005012851000A03E12751F00B5D
:1061400007E0010E120005012851000A01E0010ECE
:10615000120029C500F12AC501F12BC502F12CC599
:1061600003F125C504F126C505F127C506F128C5AB
:1061700007F14BEC2AF003BF12008FEC30F0D8A4EB
:1061800021EF31F0899A400EC76E200EC66E9E96A2
:10619000C69E060EC96EFF0E9EB602D0E82EFCD734
:1061A000898A899A9E96C69E020EC96EFF0E9EB679
:1061B00002D0E82EFCD79E96C69E27C5C9FFFF0ECB
:1061C0009EB602D0E82EFCD79E96C69E26C5C9FF75
:1061D000FF0E9EB602D0E82EFCD79E96C69E25C521
:1061E000C9FFFF0E9EB602D0E82EFCD79E96C69E33
:1061F000000EC96EFF0E9EB602D0E82EFCD7898A2B
:10620000899A9E96C69E050EC96EFF0E9EB602D056
:10621000E82EFCD79E96C69EC952FF0E9EB602D0AF
:10622000E82EFCD7C9B00AEF31F0898A0501200EAB
:106230002527E86A2623E86A2723E86A2823A9EFA6
:1062400030F01200899A400EC76E200EC66E9E96E0
:10625000C69E060EC96EFF0E9EB602D0E82EFCD773
:10626000898A899A9E96C69EC70EC96EFF0E9EB6F3
:1062700002D0E82EFCD7898A0501256B266B276B97
:10628000286B1200899A400EC76E200EC66E9E962D
:10629000C69E050EC96EFF0E9EB602D0E82EFCD734
:1062A0009E96C69EC952FF0E9EB602D0E82EFCD71F
:1062B000C9CF33F5898A1200899A400EC76E200E25
:1062C000C66E9E96C69EB90EC96EFF0E9EB602D0D1
:1062D000E82EFCD7898A1200899A400EC76E200EDC
:1062E000C66E9E96C69EAB0EC96EFF0E9EB602D0BF
:1062F000E82EFCD7898AFF0EE82EFED712008FEC1D
:1063000030F0D8A41200899A400EC76E200EC66ED7
:106310009E96C69E030EC96EFF0E9EB602D0E82E54
:10632000FCD79E96C69E27C5C9FFFF0E9EB602D01B
:10633000E82EFCD79E96C69E26C5C9FFFF0E9EB6C8
:1063400002D0E82EFCD79E96C69E25C5C9FFFF0E3B
:106350009EB602D0E82EFCD79E96C69EC952FF0E6E
:106360009EB602D0E82EFCD7898A0F01C950FF0AD9
:10637000D8A476EF34F00501FE0E336FEDEC2CF06F
:10638000ABC534F5ACC535F5ADC536F5AEC537F59D
:10639000AFC538F5B0C539F5B1C53AF50784B6C112
:1063A00066F1B7C167F1B8C168F1B9C169F14BC114
:1063B0004FF14CC150F14DC151F14EC152F157C195
:1063C00059F158C15AF1CEEC1FF000C13BF501C1A3
:1063D0003CF502C13DF503C13EF505015D67F8EFEF
:1063E00031F05E67F8EF31F05F67F8EF31F060672A
:1063F000FCEF31F009EF32F05DC504F15EC505F147
:106400005FC506F160C507F14BEC2AF003BF76EFDC
:1064100034F059C13FF55AC140F5B5C541F5B6C58F
:1064200042F5C3EC27F036C645F537C646F50601FA
:10643000406722EF32F0416722EF32F0426722EFED
:1064400032F0436726EF32F037EF32F046EC2BF0B4
:106450004CEC2BF036C600F137C601F140C604F112
:1064600041C605F14BEC2AF003AF76EF34F00101A1
:10647000036B026B1AC600F11BC601F101AF45EFB9
:1064800032F0FF0E026FFF0E036F0101076B066B08
:106490001CC604F11DC605F105AF53EF32F0FF0E27
:1064A000066FFF0E076F50EC2AF00101076B066BB9
:1064B0001EC604F11FC605F105AF63EF32F0FF0EF3
:1064C000066FFF0E076F50EC2AF00101076B066B99
:1064D00020C604F121C605F105AF73EF32F0FF0EBF
:1064E000066FFF0E076F50EC2AF0D89001010333BE
:1064F000023301330033D8900101033302330133F7
:10650000003300C147F501C148F50101036B026B7F
:1065100022C600F123C601F101AF93EF32F0FF0E66
:10652000026FFF0E036F0101076B066B24C604F1B7
:1065300025C605F105AFA1EF32F0FF0E066FFF0E85
:10654000076F50EC2AF00101076B066B26C604F1B9
:1065500027C605F105AFB1EF32F0FF0E066FFF0E53
:10656000076F50EC2AF00101076B066B28C604F197
:1065700029C605F105AFC1EF32F0FF0E066FFF0E21
:10658000076F50EC2AF0D890010103330233013336
:106590000033D8900101033302330133003300C1CB
:1065A00049F501C14AF50101036B026B2AC600F1EE
:1065B0002BC601F101AFE1EF32F0FF0E026FFF0ECB
:1065C000036F0101076B066B2CC604F12DC605F1A4
:1065D00005AFEFEF32F0FF0E066FFF0E076F50ECC6
:1065E0002AF00101076B066B2EC604F12FC605F1D8
:1065F00005AFFFEF32F0FF0E066FFF0E076F50EC96
:106600002AF00101076B066B30C604F131C605F1B3
:1066100005AF0FEF33F0FF0E066FFF0E076F50EC64
:106620002AF0D89001010333023301330033D890AC
:106630000101033302330133003300C14BF501C1C3
:106640004CF50101036B026B02C600F103C601F1B8
:1066500001AF2FEF33F0FF0E026FFF0E036F01014A
:10666000076B066B04C604F105C605F105AF3DEFE7
:1066700033F0FF0E066FFF0E076F50EC2AF001019A
:10668000076B066B06C604F107C605F105AF4DEFB3
:1066900033F0FF0E066FFF0E076F50EC2AF001017A
:1066A000076B066B08C604F109C605F105AF5DEF7F
:1066B00033F0FF0E066FFF0E076F50EC2AF0D890F4
:1066C00001010333023301330033D8900101033356
:1066D00002330133003300C14DF501C14EF5010114
:1066E000036B026B0AC600F10BC601F101AF7DEF2F
:1066F00033F0FF0E026FFF0E036F0101076B066B95
:106700000CC604F10DC605F105AF8BEF33F0FF0E9B
:10671000066FFF0E076F50EC2AF00101076B066B46
:106720000EC604F10FC605F105AF9BEF33F0FF0E67
:10673000066FFF0E076F50EC2AF00101076B066B26
:1067400010C604F111C605F105AFABEF33F0FF0E33
:10675000066FFF0E076F50EC2AF0D890010103334B
:10676000023301330033D890010103330233013384
:10677000003300C14FF501C150F50101036B026BFD
:1067800012C600F113C601F101AFCBEF33F0FF0EDB
:10679000026FFF0E036F0101076B066B14C604F155
:1067A00015C605F105AFD9EF33F0FF0E066FFF0EEA
:1067B000076F50EC2AF00101076B066B16C604F157
:1067C00017C605F105AFE9EF33F0FF0E066FFF0EB8
:1067D000076F50EC2AF00101076B066B18C604F135
:1067E00019C605F105AFF9EF33F0FF0E066FFF0E86
:1067F000076F50EC2AF0D8900101033302330133C4
:106800000033D8900101033302330133003300C158
:1068100051F501C152F507940501210E326F899A95
:10682000400EC76E200EC66E9E96C69E060EC96EA0
:10683000FF0E9EB602D0E82EFCD7898A899A9E96D2
:10684000C69E020EC96EFF0E9EB602D0E82EFCD781
:106850009E96C69E27C5C9FFFF0E9EB602D0E82EA3
:10686000FCD79E96C69E26C5C9FFFF0E9EB602D0D7
:10687000E82EFCD79E96C69E25C5C9FFFF0E9EB684
:1068800002D0E82EFCD725EE33F0322F02D054EFA1
:1068900034F09E96C69EDECFC9FFFF0E9EB602D094
:1068A000E82EFCD745EF34F0898A899A9E96C69ED9
:1068B000050EC96EFF0E9EB602D0E82EFCD79E963E
:1068C000C69EC952FF0E9EB602D0E82EFCD7C9B0B4
:1068D0005FEF34F0898A0501200E2527E86A262318
:1068E000E86A2723E86A282337EC29F0120021C53B
:1068F00000F122C501F123C502F124C503F1899AF3
:10690000400EC76E200EC66E9E96C69E0B0EC96EBA
:10691000FF0E9EB602D0E82EFCD79E96C69E02C100
:10692000C9FFFF0E9EB602D0E82EFCD79E96C69EEB
:1069300001C1C9FFFF0E9EB602D0E82EFCD79E967D
:10694000C69E00C1C9FFFF0E9EB602D0E82EFCD73E
:106950009E96C69EC952FF0E9EB602D0E82EFCD768
:1069600025EE33F00501200E326F9E96C69EC95269
:10697000FF0E9EB602D0E82EFCD7C9CFDEFF322F25
:10698000B5EF34F0898A1200899A400EC76E200E46
:10699000C66E9E96C69E900EC96EFF0E9EB602D023
:1069A000E82EFCD79E96C69E000EC96EFF0E9EB6C0
:1069B00002D0E82EFCD79E96C69E000EC96EFF0E32
:1069C0009EB602D0E82EFCD79E96C69E000EC96EDB
:1069D000FF0E9EB602D0E82EFCD79E96C69EC952E8
:1069E000FF0E9EB602D0E82EFCD7C9CF2DF59E969D
:1069F000C69EC952FF0E9EB602D0E82EFCD7C9CF64
:106A00002EF5898A120037EC29F0B5C5E8FFD708C2
:106A100002E337EC29F0B5C5E8FFC80802E337EC1C
:106A200029F0B5C5E8FFB90802E337EC29F0B5C590
:106A3000E8FFAA0802E337EC29F0B5C5E8FF9B0898
:106A400002E337EC29F095EC2DF05CEC31F0F29C90
:106A5000F29E8B94C69AC290898C9482948C720E0A
:106A6000D36ED3A4FED789968A909390FF0EE8CF79
:106A700000F0E82EFED7002EFCD78150F294F29A57
:106A80009E909D909E929D92F298F292F290F28644
:066A9000F28E0300FF007E
:10BF0000E844F926000C160C2B0C3F0C520C640C68
:10BF1000760C860C960CA50CB30CC10CCF0CDC0C6B
:06BF2000E80CF40C000C1B
:00000001FF
